:020000040800F2
:1000000040150020E9010008991D0008411D000865
:10001000951D0008ED160008FF34000800000000E0
:10002000000000000000000000000000132E000887
:10003000E517000800000000B1290008252F00087E
:10004000030200080302000803020008030200087C
:100050000302000803020008E91700080302000871
:10006000030200080302000803020008030200085C
:10007000030200080302000803020008030200084C
:10008000030200080302000803020008030200083C
:10009000030200080302000803020008030200082C
:1000A000030200080302000803020008030200081C
:1000B00003020008892F0008BD3000080302000871
:1000C00003020008030200080302000803020008FC
:1000D00003020008DD3200080302000803020008E2
:1000E00003020008030200080302000800F002F8FF
:1000F00000F06AF80AA090E8000C82448344AAF158
:100100000107DA4501D100F05FF8AFF2090EBAE855
:100110000F0013F0010F18BFFB1A43F0010318473B
:100120008C760000AC7600000A444FF0000C10F80A
:10013000013B13F0070408BF10F8014B1D1108BF65
:1001400010F8015B641E05D010F8016B641E01F805
:10015000016BF9D113F0080F1EBF10F8014BAD1C55
:100160000C1B09D16D1E58BF01F801CBFAD505E073
:1001700014F8016B01F8016B6D1EF9D59142D6D3CD
:10018000704700000023002400250026103A28BFF5
:1001900078C1FBD8520728BF30C148BF0B607047F9
:1001A000662905F08685642900F07C800020704770
:1001B0001FB500F0E5FB04000020002104F012FD53
:1001C000E0601FBD10B510BD00F0DEFC1146FFF76A
:1001D000EFFF03F091FF00F0FCFC03B4FFF7F2FF28
:1001E00003BC03F00FFA00000948804709480047A4
:1001F000FEE7FEE7FEE7FEE7FEE7FEE7FEE7FEE7D7
:10020000FEE7FEE704480549054A064B7047000033
:10021000292F0008ED000008400F002040150020A5
:100220004011002040110020704700000FB41CB5A1
:10023000074B06AA7B4469460090059800F087FBAF
:100240000020694600F096FB1CBC5DF814FB000022
:100250003D07000070B5044685690068C10601D5F8
:10026000302600E02026C00707D070BDD4E9012168
:1002700030469047206A401C20626D1EF6D570BD46
:1002800070B5044685690078C00707D170BDD4E910
:10029000012120209047206A401C20626D1EF6D567
:1002A00070BD00002DE9F041064600241068752954
:1002B000314616A510D0AFF30080002802DA404284
:1002C00013A507E031688A0701D512A502E04907A6
:1002D00004D511A5012401E0AFF3008000210A221A
:1002E00006F1240709E0B0FBF2FCB0FBF2F302FBDD
:1002F0001C00303078541846491C0028F3D123469E
:100300002A463046BDE8F04100F0B3B800000000D6
:100310002D0000002B000000200000002DE9F05F00
:10032000894604464FF0000ADFF824B1FB44C0F8C8
:1003300020A02046E168884700287DD0252806D0E7
:10034000D4E901219047206A401C2062F1E7002592
:100350005F462046E16888472028064607DB312EA5
:1003600005D2B81910F8200C08B10543F1E7A80729
:1003700001D525F00405C4F81CA00027C4F818A076
:100380002A2E09D0304603F036F938B304EB87083B
:10039000303EC8F8186019E059F8041B204604EBF9
:1003A00087029161E1688847012F064618D1E0690C
:1003B000002820DA25F020051DE0D8F8180000EB11
:1003C000800006EB40003038C8F818002046E1688D
:1003D0008847064603F00FF90028EED1012F0AD016
:1003E0002E2E08D12046E16888477F1C0646022F42
:1003F00045F02005C4DBA069002803DA404245F03F
:100400000105A061E80701D025F01005A6B1A6F10D
:100410004100192802D8203645F400654A46314685
:10042000204625604D46FFF7BBFE60B1012807D08E
:10043000ED1D25F0070000E007E000F1080978E76E
:1004400005F1040975E730467AE7206ABDE8F09FB8
:1004500090730000704770477047704710B500F008
:1004600093FA006810BD10B5044600F08DFA0460E0
:1004700010BD2DE9F0470D4699469246044600F11D
:1004800024080168880604D5E06921F01001216084
:1004900000E00120A84201DD471B00E00027A16920
:1004A0007A1902EB0900081AA0612078C00602D46C
:1004B0002046FFF7CFFE002608E0D4E901211AF814
:1004C00006009047206A401C761C20624E45F4DBF3
:1004D0002078C0060AD52046FFF7BCFE06E0D4E926
:1004E000012130209047206A401C2062381EA7F16D
:1004F0000107F4DC07E0D4E9012118F80500904772
:10050000206A401C2062281EA5F10105F3DC20466C
:10051000FFF7B6FE2078000602D50220BDE8F0877E
:100520000120FBE770472DE9FF4F0C461E464FF0B8
:10053000FF378BB0D2E90001DDF860800A908A466F
:10054000C1F30A5505B93D46002108464FF00000A9
:10055000BAF1000F00F4400005DA00EB80004FF420
:10056000400101EA50004FEA9059B9F1010F00DD56
:10057000B9460A9850EA4A000ED044F61050A5F247
:10058000FF3545432F14B8F1000F1ED07542291EC8
:100590001EDDC9F100021CE0B8F1010F4FF00000B0
:1005A00001D0302103E0F24305E02154401CB04269
:1005B000FBDB30460022002121540B99C1F8088052
:1005C000C1E900200FB0BDE8F08FBD1B6D1CDEE758
:1005D0004A4600DA694206A800F060FA06AB93E8E2
:1005E000070003AB83E8070050460A9900F03AFB86
:1005F0008DE80700A0F500501F3800900398002DEB
:100600000ADD42F21F014A460844002303A9039071
:10061000684600F0A3FD09E0A0F500504A461F38E7
:10062000002303A90390684600F0ADFD8DE80700A4
:100630000004000C03D04FF0FF30410800E01046EA
:10064000B8F1000F03D00022009215461EE0751E7F
:1006500005D400F09DF9303262556D1EF9D5B346D0
:100660000122084302D000227F1C04E020783028B9
:1006700001D100227F1E002A099784D01DE0112D90
:1006800007DA00F085F9303262556D1C50EA01023C
:10069000F5D1084302D00098C8B10EE00021681ED1
:1006A00005E0235C625C63542254401E491C814275
:1006B000F7DBAB46A81B401E0990002004F80B0096
:1006C0000B98099AC0F80880C0E9002B7AE7112638
:1006D0004FF0000857E72DE9F04F88460446D21D39
:1006E00022F0070191B0D1E90001CDE90A0102F041
:1006F00008FF02460B98C00F01D02D2007E02068AC
:10070000810701D52B2002E0202101EAC000032A45
:10071000099001D0072A05DB03464146204600F038
:100720007DF90BE12078800601D5E06900E0062024
:10073000B8F1650F814606D0B8F1660F18D0B8F150
:10074000670F70D131E00020B9F1110F009001DB8B
:10075000112301E009F101030AAA01A90CA8FFF77E
:10076000E2FEDDE90C70002609F10105834647E051
:1007700001204B4600904FF000470AAA01A90CA89F
:10078000FFF7D1FEDDE90DB00C995D46002610B9EA
:1007900009F101000D18B9EB050003D4C0F1FF36D3
:1007A00009F10105A5EB09002BE0B9F1010F01DA10
:1007B0004FF001090020B9F1110F0090484601DD0A
:1007C000112300E003460AAA01A90CA8FFF7ABFE1B
:1007D000DDE90C704D4600268346207800070AD4D8
:1007E000AB4500DA5D4601A8012D04DD411911F881
:1007F000011C302907D04F4502DA17F1040F04DA43
:10080000012082460FE06D1EEEE7002F02DCED1B9B
:100810003E4403E0781CA84200DD7D1CB81B00F1BB
:10082000010A4FF000472078000703D4AA4501DBF6
:100830004FF0FF3A0021B7F1004F0DF143088DF85A
:10084000431024D002202B23002F01DA7F422D23D6
:100850000A21021EA0F1010000DC5FB197FBF1FC50
:1008600097FBF1F201FB1C7C17460CF1300C08F8E9
:1008700001CDEEE7A8F1010003702188090501D53B
:10088000452100E06521A0F1010800F8011C09984C
:100890000FA9A1EB0807FF1D00B10120411901EBD1
:1008A000EA70A1693844081A401EA0612078C00689
:1008B00002D42046FFF7CEFC099828B1D4E90121E3
:1008C0009047206A401C20622078C00622D520462E
:1008D000FFF7C0FC1EE0002E04DBB34502DD01A8DB
:1008E000805D00E03020D4E901219047206A401C5F
:1008F0002062761CAAF101005FEA000A0AD100F02A
:100900003FF8C0680168405CD4E901219047206A43
:10091000401C2062281EA5F10105DCDC07E0D4E9BB
:10092000012118F8010B9047206A401C2062381EF4
:10093000A7F10107F3DC2046FFF7A2FC032011B06A
:1009400041E6000001694A1C02610878704700B561
:100950008FB0CDE901310021059105497944CDE9F8
:10096000031011466846FFF7D9FC0FB000BD000028
:10097000E5FFFFFF0A6802F8010B0A6070470000FC
:1009800000487047FC0E002000487047DC0E002035
:1009900030B5B0F10A024FEA900E71F100034EEA51
:1009A000817EB0EB0E0061EB91014FEA101E4EEA22
:1009B000017E10EB0E0041EB11114FEA102E4EEAB2
:1009C000016E10EB0E0041EB11214FEA104E4EEA82
:1009D000014E10EB0E0041EB1141401841F10001B6
:1009E0004FEAD00040EA41704FEAD10110EB800598
:1009F0004FEA810444EA907444EB01046D1944EB1E
:100A00000404521BA3414FF0000348BF0A3200D533
:100A100030BD401C41F1000130BD00002DE9F04126
:100A20001F46044603260168072A01F4006004DB20
:100A300008B116A505E016A503E008B115A500E06C
:100A400015A521F010002060A069C01EA0610FB1A3
:100A5000401EA0612046FFF7FDFB4FB1D4E9012104
:100A600038469047206A401C2062C01C206206E085
:100A7000206AFAE7D4E9012115F8010B9047761EA8
:100A8000F8D22046FFF7FCFBBDE8F0814E414E0056
:100A90006E616E00494E4600696E66002DE9F047B2
:100AA000814616468AB0354878440DC88DE80D0059
:100AB00032487844801C03AC0DC884E80D0041F630
:100AC0009B300844372190FBF1F290FBF1F5A5F142
:100AD000800501FB12041B3C02D56442012000E0AA
:100AE0000020DFF898A080460027FA44AAF1BE0A49
:100AF0000EE0E0070AD03246684607EB47010123C3
:100B00000AEB810100F03FFB8DE8070064107F1CB9
:100B1000002CEED1194F7F44AE3F19E0E80715D005
:100B200007EB04100DF1180A90E80E008AE80E0099
:100B3000C068F04201D1981908903246012306A9F5
:100B400003A800F020FB03AB83E807006D10641CD2
:100B5000002DE3D14FF0010332466946B8F1000F92
:100B600003A802D000F0FAFA01E000F00CFBC9E99A
:100B70000001C9F808200AB0BDE8F087E86C000061
:100B800000487047DC0E00207546FFF7F9FFAE46BF
:100B900005006946534620F00700854618B020B589
:100BA000FFF730FBBDE820404FF000064FF0000794
:100BB0004FF000084FF0000B21F00701AC46ACE805
:100BC000C009ACE8C009ACE8C009ACE8C0098D4672
:100BD000704710B50446AFF300802046BDE81040D2
:100BE000FFF7FBBA4FF0013C50F8042B51F8043BDF
:100BF0009A4221D1A2EB0C03934313EACC1317D1F1
:100C000050F8042B51F8043B9A4215D1A2EB0C0387
:100C1000934313EACC130BD150F8042B51F8043B47
:100C20009A4209D1A2EB0C03934313EACC13DBD015
:100C30004FF00000704700BFD01A01BAB1FA81F13D
:100C400001F0180122FA01F0CB40C1F12001DBB222
:100C5000C0B2C01A2CFA01F3D11A914311EAC311A0
:100C6000E6D170475FEA400C08BF91F0000F4FEAF1
:100C70008C234FEAC12243EA51514FEA1C5018BF5E
:100C800000F5F0404FEA300018BF41F000415FEA44
:100C90006C5C00F02980BCF1FF3F08BF40F0804051
:100CA0007047130C06BF12044FF0100C4FF0000CED
:100CB000130E04BF12020CF1080C130F04BF120133
:100CC0000CF1040C930F04BF92000CF1020CD30F33
:100CD00004BF52000CF1010C11464FF00002A0F1CC
:100CE0001F00A0EB0C00704711F0004F08BF7047C9
:100CF00031F000413FF4D5AF0B0C06BF09044FF0B3
:100D0000100C4FF0000C0B0E04BF09020CF1080C84
:100D10000B0F04BF09010CF1040C8B0F04BF8900F9
:100D20000CF1020CCB0F04BF49000CF1010CCCF10B
:100D30002003A0EB0C0022FA03F302FA0CF241EAC2
:100D4000030100F10100704720F07F4C80EA0300AE
:100D500023F07F47ACEB070303F57C5300F0004022
:100D600003F1FF032DE980494FEA154B09B44FEA1F
:100D7000144325EA0B4E24EA03480FF2042606EB3F
:100D8000132749083E785FEA320203FB0667C7F57E
:100D9000000707FB06F64FEA54374FEAD64606F13E
:100DA000020607FB066CCCF1005C4FEA1C472CEAFC
:100DB000074C07FB06F40CFB06F504EB15464FEA5F
:100DC000961634BF00204FF000404FEAD13706FBA3
:100DD00007FC4FEA1C4C0CFB0BF7D21B03FB0CF778
:100DE00061EB07010CFB0EF7B0EB074072EB17420B
:100DF0000CFB08F734BFA2EB0742B2EB074261EBF2
:100E000017414FEA0C444FEA910706FB07FC4FEAF3
:100E10001C4C0CFB0BF7B0EBC74072EB573203FBDB
:100E20000CF734BFA2EBC742B2EBC74261EB5731BC
:100E30000CFB0EF7B0EBC70072EB57720CFB08F718
:100E400034BFA2EBC702B2EBC70261EB5771039F3D
:100E50004FEA816141EA921104EBCC044FEAD137A9
:100E60004FEA826206FB07FC42EA90124FEA80607A
:100E70004FEA1C4C0CFB0BF7D21B03FB0CF761EB8E
:100E800007010CFB0EF7B0EB074072EB17420CFBAF
:100E900008F734BFA2EB0742B2EB074261EB174100
:100EA0004FEA8C554FEA910704EB9C2406FB07FCA4
:100EB0004FEA1C4C0CFB0BF7B0EBC74072EB573200
:100EC00003FB0CF734BFA2EBC742B2EBC74261EBA6
:100ED00057310CFB0EF7B0EBC70072EB57720CFBEF
:100EE00008F734BFA2EBC702B2EBC70261EB577140
:100EF00015EB4C254FEA816141EA92114FEA82627B
:100F00004FEAD13742EA901206FB07FC44F1000495
:100F10004FEA80604FEA1C4C0CFB0BF7D21B03FB23
:100F20000CF761EB07010CFB0EF7B0EB074072EB1F
:100F300017420CFB08F734BFA2EB0742B2EB0742A3
:100F400061EB174115EB1C154FEA813141EA9241E3
:100F50004FEA823242EA90424FEA80304FEA0C7602
:100F600044F1000448EA03434EEA0B484FF0000EF8
:100F7000B2EB080C71EB030724BF624639464EEB17
:100F80000E0E4FF0000B0018524149414BEB0B0B7A
:100F9000B2EB080C71EB03077BF1000B24BF624638
:100FA00039464EEB0E0E4FF0000B001852414941EE
:100FB0004BEB0B0BB2EB080C71EB03077BF1000B57
:100FC00024BF624639464EEB0E0E51EA020718BFA7
:100FD00046F0010616EB0E7655F1000254F10001C1
:100FE00003D5BDE88901BDE80088BDE88901BDE8F9
:100FF0000048B619524141EB0101A3F101037047CA
:1010000080807F7E7D7C7B7A797877767675747345
:10101000727171706F6E6E6D6C6C6B6A6A69686804
:10102000676666656464636362616160605F5F5E9A
:101030005E5D5D5C5C5B5B5A5A5959585857575610
:101040005655555554545353525252515150505075
:101050004F4F4F4E4E4D4D4D4C4C4C4B4B4B4A4AC7
:101060004A4949494848484747474746464645450B
:101070004544444444434343434242424241414144
:10108000002B9C4630D477002BD01CB54FEA370795
:1010900003B44FF010004FF01001BAF1000F06D06A
:1010A000BCF1000FDCBF40F0080040F008014FF039
:1010B00000000FBCBDE810400BF1010BBBF1010FAC
:1010C00008BF5FEA170722BF12F1010211F1010107
:1010D0004FF0004143F1000300F0004043EA0000FC
:1010E0007047F9D35708D0E746EA064613F1400F98
:1010F0004FEA16461FDD13F1200FDFBF16430A46E5
:10110000002120335B42BED0C3F1200746EA0646E9
:1011100002FA07F74FEA164646EA0706C3F1200728
:1011200022FA03F201FA07F721FA03F14FF0000364
:1011300042EA0702A7E746EA020646EA06464FEAFF
:10114000164646EA0106BCBF46EA0646360C4FF094
:1011500000034FF000024FF0000194E72DE9804CAE
:101160009A46934670B491E8380007C831EA400CBB
:1011700048BF34EA430C03D5FFF7E6FDFFF780FFD5
:10118000F0BCBDE8008C2DE9804C9A46934670B4C3
:1011900091E8380007C810F0804F08BF13F0804F67
:1011A00003D100F005F8FFF76BFFF0BCBDE8008C41
:1011B00020F07F4780EA030023F07F4C07EB0C030D
:1011C000A3F57C5300F00040A3F1FE0392F0000F62
:1011D00000F0B38095F0000F00F077802DE9014911
:1011E0004FEA11404FEA144621EA004800FB06FC92
:1011F00024EA064708FB06F607FB08F800FB07F79A
:1012000018EB06484CEB164C4FEA124B18EB07480C
:101210004FEA15464CEB174022EA0B4E0BFB06FC3F
:1012200025EA06470EFB06F607FB0EFE0BFB07F74B
:101230001EEB064E4CEB164C4FF000061EEB074E15
:101240004CEB174B18EB0B0840F1000018EB0E0BA2
:1012500058EB000840F100008F1A4FF000013CBF2E
:10126000C943661B14BFB5EB040C00213CBFC94346
:10127000F61B4FEA17444EEA8E0E27EA04454FEA62
:101280001C4704FB07622CEA074C05FB07F70CFB25
:1012900005F604FB0CFC16EB074642EB174216EB77
:1012A0000C4642EB1C421BEB060658EB0202414186
:1012B00046EA9E0601D5BDE80189B619524141EBC7
:1012C0000101A3F10103BDE801894FEA14454FEA8A
:1012D000114724EA054621EA074C05FB07F406FB03
:1012E00007F70CFB06F105FB0CFC11EB074144EB87
:1012F00017444FEA124711EB0C4144EB1C4422EA1D
:10130000074C05FB07F206FB07F70CFB06F605FB8F
:101310000CFC16EB074642EB174216EB0C4642EB71
:101320001C456A1854F1000148BF7047B619524174
:1013300041EB0101A3F10103704795F0000F37D095
:101340004FEA11424FEA144721EA024624EA074CC9
:1013500002FB07F106FB07F70CFB06F402FB0CFC93
:1013600014EB074441EB17414FEA154714EB0C44CB
:1013700041EB1C4125EA074C02FB07F506FB07F78A
:101380000CFB06F602FB0CFC16EB074645EB17457B
:1013900016EB0C4645EB1C42121951F1000148BFF7
:1013A0007047B619524141EB0101A3F101037047A7
:1013B0004FEA14454FEA114724EA054621EA074C53
:1013C00005FB07F106FB07F70CFB06F24FF00006E2
:1013D00005FB0CFC12EB074241EB174112EB0C42F0
:1013E00051EB1C4148BF7047921841EB0101A3F13A
:1013F0000103704721B1826842F00102826003E07C
:10140000826822F0010282607047000010B5044635
:101410001248844208D10121401501F0F7FA002159
:10142000601501F0F3FA17E00D48844208D101215C
:10143000001501F0EBFA0021201501F0E7FA0BE0AE
:101440000848844208D10121C80301F0DFFA0021D5
:101450004FF4004001F0DAFA10BD00000024014012
:1014600000280140003C0140014600208A6802F04B
:1014700004020AB1012000E0002070470146C86C58
:1014800080B270470246002013680B400BB1012068
:1014900000E000207047014600208A6802F0080240
:1014A0000AB1012000E000207047000030B502467C
:1014B0000020002350680F4C20400D790C6844EA4E
:1014C00005242043506090680B4C2040D1E9025421
:1014D0002C434D7944EA450420439060D06A20F4BF
:1014E00070000C7C641EE4B2234340EA0350D062D7
:1014F00030BD0000FFFEF0FFFDF7F1FFF0B5044640
:101500000D4600200021092D11DDE068A5F10A0635
:1015100006EB4607072606FA07F18843A5F10A06F7
:1015200006EB460603FA06F10843E0600CE020698A
:1015300005EB4507072606FA07F1884305EB450644
:1015400003FA06F108432061072A0FDA606B561E82
:1015500006EB86071F2606FA07F18843561E06EBA0
:10156000860605FA06F10843606322E00D2A0FDAC9
:10157000206BD61F06EB86071F2606FA07F1884365
:10158000D61F06EB860605FA06F10843206310E035
:10159000E06AA2F10D0606EB86071F2606FA07F1A0
:1015A0008843A2F10D0606EB860605FA06F108430C
:1015B000E062F0BD816841F008018160704721B1AF
:1015C000826842F4A002826003E0826822F4A002F2
:1015D00082607047816841F00401816070470000BB
:1015E00000B587B00121042001F000FA5420ADF8C5
:1015F000180003208DF81A0000208DF81B0006A9A2
:101600002A4800F00BFA4FF48070ADF8180004205F
:101610008DF81B0006A9254800F000FA01214802B8
:1016200001F0E4F94FF4004001F0C4F92048FFF75D
:10163000EDFE002001908DF808008DF809004FF4B0
:10164000602003900020049001208DF8140001A96F
:101650001748FFF72BFF0723012202211448FFF749
:101660004DFF0723012204211148FFF747FF0723FD
:10167000012206210E48FFF741FF01210C48FFF728
:10168000B9FE0B48FFF796FF00BF0948FFF703FFBD
:101690000028FAD10648FFF79DFF00BF0448FFF776
:1016A000E3FE0028FAD107B000BD000000080140A9
:1016B0000024014008B50121082001F097F94FF4FA
:1016C0000070ADF8000010208DF8030003208DF8A5
:1016D00002006946044800F0A1F94FF40071024885
:1016E00000F079FA08BD0000000C014000BFFEE7E1
:1016F000F8B5054600246DE0C4EBC400374901EBA2
:10170000800005EB0413D3E901621968DB68C0E9C6
:101710000162C3600160C4EBC401304A02EB810185
:10172000C868012101F062F9C4EBC4002B4901EB48
:10173000800000892DF82400C4EBC40011F82000BB
:10174000694601EB8401C8706A4602EB8401C4EB70
:10175000C402224B03EB8202506800F05FF90120C3
:10176000C4EBC4011D4A02EB810108740021C4EBE3
:10177000C40002EB80004174C4EBC40002EB8000A3
:101780008174C4EBC400114611F82000482806D12A
:101790000021C4EBC40002EB8000C17406E001210B
:1017A000C4EBC4000D4A02EB8000C1740021C4EBFD
:1017B000C4000A4A02EB80000175C4EBC40002EBCE
:1017C000800041750649C4EBC40002EB80008161D2
:1017D000601CC4B2012C8FDBF8BD0000E8090020BA
:1017E000851D00087047000010B5012001F044FF7E
:1017F00001200A4908800A4800680A49D1F80C11FA
:10180000884203D106200549488002E007200349A9
:101810004880012000F008F810BD000058000020AA
:101820000081214200802142014908607047000088
:1018300014040140002123498279002A3AD00A4643
:10184000126803689A430B461A600A1D12680368FF
:101850009A430B1D1A60027911440A6803681A43FF
:101860000A60184A0832126803689A43154B083315
:101870001A601A1D126803689A43124B0C331A60DF
:101880004279102A0ED11A1F126803681A430D4BB1
:1018900008331A601A1D126803681A43094B0C3387
:1018A0001A600DE00749427911440A6803681A4337
:1018B0000A6005E0027911440A6803689A430A60E5
:1018C000704700000004014030B5044604254FF481
:1018D000302000F06FF80546042D17D10C48006940
:1018E00040F002000A49086108464461006940F07E
:1018F000400008614FF4302000F05CF805460448D1
:10190000006941F6FD71084001490861284630BD73
:101910000020024004200B49C96801F0010109B10F
:1019200001200EE00749C96801F0040109B1022055
:1019300007E00449C96801F0100109B1032000E083
:1019400004207047002002400348006940F08000F6
:1019500001490861704700000020024070B504464C
:101960000D460426F00200F025F80646042E11D19B
:101970000948006940F00100074908612580F0022C
:1019800000F018F806460448006941F6FE71084068
:1019900001490861304670BD0020024002480349F9
:1019A00048600348486070472301674500200240B3
:1019B000AB89EFCD00B502460423FFF7ABFF03462A
:1019C00003E0FFF7A7FF0346521E012B01D1002AB7
:1019D000F7D102B90523184600BD000030B500223A
:1019E0008B071C0F0F2303FA04F20B4B8C1053F8D8
:1019F00024309343084C8D1044F8253023468C1036
:101A000053F824308C07240F00FA04F42343024CCB
:101A10008D1044F8253030BD080001402DE9F0411B
:101A2000024600250026002000230024002791F80C
:101A300003C00CF00F0591F803C00CF0100CBCF1C2
:101A4000000F03D091F802C04CEA050591F800C0E0
:101A5000BCF1000F31D0146800202BE04FF0010CD6
:101A60000CFA00F3B1F800C00CEA03069E4220D144
:101A700083004FF00F0C0CFA03F7BC4305FA03FC8C
:101A80004CEA040491F803C0BCF1280F06D14FF0D2
:101A9000010C0CFA00FCC2F814C00AE091F803C073
:101AA000BCF1480F05D14FF0010C0CFA00FCC2F854
:101AB00010C0401C0828D1D31460B1F800C0BCF19C
:101AC000FF0F34DD546800202EE000F1080C4FF0C9
:101AD000010808FA0CF3B1F800C00CEA03069E42B4
:101AE00021D183004FF00F0C0CFA03F7BC4305FA29
:101AF00003FC4CEA040491F803C0BCF1280F05D1A3
:101B000000F1080C08FA0CF8C2F8148091F803C030
:101B1000BCF1480F07D100F1080C4FF0010808FA9A
:101B20000CF8C2F81080401C0828CED35460BDE8E1
:101B3000F0810000F0B50A460023002400210025B2
:101B400000F00046B6F1004F02D11D4EF16901E0F0
:101B50001B4E7168C0F3034583B200F44016B6F51E
:101B6000401F08D121F07061154E766826F070662E
:101B7000134F7E6012E000F48016B6F5801F06D188
:101B8000032606FA05F4A14341F0706106E0460D14
:101B9000360103FA06F6B14341F0706122B1460DF9
:101BA000360103FA06F6314300F00046B6F1004F65
:101BB00002D1034EF16101E0014E7160F0BD000001
:101BC000000001400246002093680B400BB1012049
:101BD00000E00020704741617047016170470000DC
:101BE00010B504460723012221460948FFF786FC69
:101BF00001210748FFF7E3FC00BF02210448FFF77B
:101C000041FC0028F9D00248FFF738FC10BD000065
:101C1000002401402DE9F04107460C46002500262E
:101C200008E03846FFF7DCFF0544052001F04AFDD7
:101C3000701CC6B2A642F4DBB5FBF4F080B2BDE87E
:101C4000F081000070B500242DE0C4EBC4001749FA
:101C500001EB8000007C00B923E0C4EBC400134911
:101C600001EB8005C4EBC40001EB8000866995E8B8
:101C70000F00B047C4EBC4010C4A02EB8101C97CE0
:101C8000884206D10121C4EBC40002EB80008174BC
:101C900006E00021C4EBC400044A02EB800081741A
:101CA00000BF601CC4B2012CCFDB70BDE80900206E
:101CB00000B589B00121084600F088FE012104200A
:101CC00000F094FE0120ADF8200018208DF82300CC
:101CD00003208DF8220008A91748FFF79FFE174838
:101CE0000088401E80B2ADF8180040F2CF20ADF859
:101CF00014000020ADF81A00ADF8160005A94FF049
:101D0000804001F099FA6020ADF804000120ADF8A0
:101D100006000020ADF80C0001A94FF0804001F052
:101D200033FA0821C80601F07BFA0121880701F087
:101D300004FA09B000BD0000000801409005002031
:101D400000BFFEE71FB50C4B0FCB8DE80F0001F075
:101D5000DFFC6846FFF7CCFC0121084600F046FE98
:101D600001210648FFF7E6FE0548406820F0200004
:101D7000034948601FBD0000A85D00080002300054
:101D8000002004E01FB5BDF808100198FFF71AFF06
:101D900004B010BD00BFFEE77047000070B5002121
:101DA00000230F22C47804B3154C246804F4E064C3
:101DB000C4F5E064210AC1F10403CA40447804FA7E
:101DC00003F184781440214309010E4C0678A15593
:101DD000047804F01F050124AC4005786D11AD00B6
:101DE00005F1E025C5F8004109E0047804F01F057D
:101DF0000124AC40044D0678761145F8264070BDAC
:101E00000CED00E000E400E080E100E00249014365
:101E1000024A1160704700000000FA050CED00E076
:101E200070B5002419E004F1B001C8B2002100F03F
:101E30006FFB0021084600F06BFB0021102000F032
:101E400067FB002505E00121002000F061FB681C14
:101E5000C5B2802DF7DB601CC4B2082CE3DB70BD7B
:101E6000F0B5144600267F2801DC3F2900DDF0BDD7
:101E70000B46CF1701EB5777FF10C7F10707FAB2F0
:101E8000CF1701EB5777FF10A1EBC707FDB2C5F1E4
:101E900007070123BB40DEB24CB10A4B03EBC00382
:101EA0009B5C3343074F07EBC007BB5408E0054B6F
:101EB00003EBC0039B5CB343024F07EBC007BB546B
:101EC00000BFD4E7040A00202DE9F04F06460C4677
:101ED00017469846A346002530E017F805904FF0C6
:101EE000000A25E009F0800028B1214630460A9A10
:101EF000FFF7B6FF09E00A9808B9012000E00020CA
:101F0000024621463046FFF7ABFF4FF6FF7000EA6E
:101F10004909601CC4B2A4EB0B010998814203D1AA
:101F20005C46701CC6B206E00AF101001FFA80FA96
:101F3000BAF1080FD6DB00BF681C85B2099908FB0F
:101F400001F0C11700EB5171B5EBE10FC5DBBDE846
:101F5000F08F00002DE9F04F07460C4690461D46D5
:101F6000A346002631E01B4800EB481010F806900D
:101F70004FF0000A23E009F0800028B12A462146EC
:101F80003846FFF76DFF08E00DB9012000E00020A2
:101F9000024621463846FFF763FF4FF6FF7000EA1E
:101FA0004909601CC4B2A4EB0B00322803D15C4683
:101FB000781CC7B206E00AF101001FFA80FABAF1F4
:101FC000080FD8DB00BF701C86B2B02ECBDBBDE89B
:101FD000F08F0000006900082DE9F04706460F4623
:101FE00090469946DDF820A034460CE03D4606E0D8
:101FF000524629462046FFF733FF681CC5B24D45BF
:10200000F6DD601CC4B24445F0DD00F0B3F8BDE875
:10201000F087000008B50121082000F0E7FC4FF42C
:102020003C40ADF8000010208DF8030003208DF82F
:10203000020069464E48FFF7F1FC4FF42C414C4832
:10204000FFF7CBFD4FF480514948FFF7C4FD4FF433
:1020500080614748FFF7C1FD642001F00DFB4FF49C
:1020600080614348FFF7B7FDC82001F005FB4FF43E
:1020700080613F48FFF7B1FD0021AE2000F048FA33
:102080000021084600F044FA0021102000F040FA38
:102090000021402000F03CFA0021812000F038FAB5
:1020A0000021CF2000F034FA0021A12000F030FA06
:1020B0000021C02000F02CFA0021A62000F028FA10
:1020C0000021A82000F024FA00213F2000F020FA8F
:1020D0000021D32000F01CFA0021084600F018FA75
:1020E0000021D52000F014FA0021802000F010FA21
:1020F0000021D92000F00CFA0021F12000F008FAAC
:102100000021DA2000F004FA0021122000F000FA89
:102110000021DB2000F0FCF90021402000F0F8F95C
:102120000021202000F0F4F90021022000F0F0F955
:1021300000218D2000F0ECF90021142000F0E8F9D6
:102140000021A42000F0E4F90021A62000F0E0F92D
:102150000021AF2000F0DCF90021AF2000F0D8F919
:10216000FFF75EFE0021084600F02AF808BD0000D7
:10217000000C014070B500241CE004F1B001C8B2AD
:10218000002100F0C5F90021084600F0C1F9002146
:10219000102000F0BDF9002508E0084901EBC50159
:1021A000085D012100F0B4F9681CC5B2802DF4DB94
:1021B000601CC4B2082CE0DB70BD0000040A0020E3
:1021C00070B504460D4605F1B001C8B2002100F01B
:1021D0009FF9102141EA1410002100F099F904F050
:1021E0000F0141F00100002100F092F970BD0000E4
:1021F0002DE9F84F80460F4616461C46BA46204643
:10220000E31704EB5373DB1021464FEAE47C04EB45
:102210005C7C4FEAEC0CA4EBCC0CBCF1000F02D0C0
:102220004FF0010C01E04FF0000C6344224604EB38
:10223000D27C4FEA6C0C03FB0CF303F0FF0BA6F10E
:102240002000C6B200254EE00C2C07D106EB46005C
:10225000274901EB8000405D009013E0102C05D170
:10226000244800EB0610405D00900BE0182C07D1CD
:1022700006EBC600204901EB8000405D009001E0C4
:10228000BDE8F88F4FF0000927E0009800F08000CB
:1022900028B1394640460A9AFFF7E2FD09E00A985C
:1022A00008B9012000E00020024639464046FFF709
:1022B000D7FD00984006000E0090781CC7B2A7EB2F
:1022C0000A00A04205D1574608F1010000F0FF08BE
:1022D00006E009F1010000F0FF09B9F1080FD4DBB5
:1022E00000BF681CC5B25D45AEDB00BFC8E700009B
:1022F000785E0008EC620008DC6800082DE9FE4FFB
:1023000006460D4617461C46DDF830A001952046CE
:10231000E21704EB5272D2102146E31704EB537319
:10232000DB10A4EBC3030BB1012300E000231A442C
:102330006243D2B200920C2C05D107EB470025492D
:1023400001EBC0090AE0102C03D1234800EB471928
:1023500004E007EBC700214901EBC0094FF000087A
:1023600032E019F808B00020029025E00BF0800060
:1023700028B1E9B2F0B25246FFF772FD0AE0BAF1B5
:10238000000F01D1012300E000231A46E9B2F0B2A8
:10239000FFF766FD4FEA4B604FEA106B681C85B291
:1023A0000198281AA04203D1019D701C86B206E054
:1023B0000298401CC0B2029002980828D6DB00BFE9
:1023C00008F1010000F0FF0800988045C9DBBDE876
:1023D000FE8F000080700008987000087876000872
:1023E0002DE9F8430546884616461F46DDF820903D
:1023F00000240BE0CDF80090325D05EB041188B2AB
:1024000010234146FFF77AFF601CC4B2BC42F1DBE7
:10241000BDE8F8832DE9FF4F81B0074691461E467F
:102420000E9D4FF0000A002439E0301B401EC1B25F
:102430000A2002F037FBB9FBF0F00A21B0FBF1F201
:1024400001FB1208BAF1000F16D1701EA04213DD75
:10245000B8F1000F0ED10120AB4605EBDB7149103E
:1024600001FB04710090C8B22B4620220299FFF7AD
:10247000BFFE12E04FF0010A0120AB4605EBDB7115
:10248000491001FB04710090C8B208F13001CAB2D2
:102490002B460299FFF7ACFE00BF601CC4B2B442E9
:1024A000C3DB05B0BDE8F08F2DE9F84306460F46C3
:1024B00015461C46DDF8208021E004EBD47149105C
:1024C000C1F18001B14202DA00263819C7B2C4F165
:1024D0004000B84204DA002006460746FFF7A0FC99
:1024E000CDF800802A78234639463046FFF780FE33
:1024F000204604EBD07106EB6101CEB26D1C28784A
:102500007E2802DC28782028D7DABDE8F88300008E
:1025100070B504460E462EB14FF400611748FFF720
:102520005CFB04E04FF400611448FFF754FB002506
:102530001BE04FF400511148FFF74DFB04F0800001
:1025400028B14FF400410D48FFF747FB04E04FF47A
:1025500000410A48FFF73FFB4FF400510748FFF7DF
:102560003CFB6006040E681CC5B2082DE1DB4FF48D
:1025700000610248FFF731FB70BD0000000C014014
:1025800008B54C484088801F05283BD2DFE800F0A2
:102590000E0319242F004848007800EB40004749FB
:1025A00001EB80004078444908702BE042480078F5
:1025B00000EB4000414901EB800080783E49087003
:1025C00020E03D48007800EB40003C4901EB8000F2
:1025D000C0783949087015E03748007800EB4000B2
:1025E000364901EB80000079334908700AE032482F
:1025F000007800EB4000314901EB800040792E4922
:10260000087000BF00BF2C48007848B92C480078FB
:1026100030B100203F237F2201460090FFF7DCFC11
:102620002548007801281ADB23480078082816DCA2
:1026300023480078012801DA012000E00020204929
:102640000978082901DD012100E00021084330B1AB
:1026500000203F237F2201460090FFF7BDFC164873
:10266000007809281ADB144800780D2816DC144875
:102670000078092801DA012000E0002010490978DB
:102680000D2901DD012100E00021084330B10020C7
:102690003F237F2201460090FFF79EFC0649097800
:1026A00001EB4101054A02EB810188688047FFF791
:1026B00061FD08BD5800002064000020B85D0008DE
:1026C000650000202DE9F0478048008803F02CF9D0
:1026D0007F4908607F48007838B1084601687E4825
:1026E00003F072FA7D4908602EE07D48407BF0B926
:1026F0007B48D0F801003230B0F5C87F07DD744860
:102700000168784803F060FA744908601CE0744975
:10271000D1F8011001F1320003F0EEF804466C48E4
:102720000168204603F050FA6C4908600CE06C49DF
:10273000D1F8010003F0E0F804466548016820463E
:1027400003F042FA6549086067496448006803F08D
:10275000FFF904D265480088654908609AE0654938
:102760005E48006803F0F4F94AD2634801684FF00C
:10277000804003F021F9824658480168504603F032
:1027800018FA80465D480168404602F049FF074656
:102790005B4801685B48006803F00EF981463946E2
:1027A00003F00AF90546584801685648006803F0E6
:1027B00003F9814649480168484603F0FDF8074699
:1027C0004D4801684548006803F0FEF981464D48D0
:1027D0000168484603F0F0F88046394602F020FFD1
:1027E0000646294602F01CFF044603F049F8474913
:1027F00008603F480068096808443D49086049E0AE
:102800003D4801684FF0804003F0D6F882463348D7
:102810000168504603F0CDF905463848016828465E
:1028200002F0FEFE80463A4801683A48006803F02C
:10283000C3F88146414603F0BFF8044636480168B4
:102840003448006803F0B8F88146244801684846D7
:1028500003F0B2F80546284801682048006803F0F4
:10286000B3F981462B480168484603F0A5F8804635
:10287000294602F0D5FE0746214602F0D1FE064663
:1028800002F0FEFF21490860194800680968084401
:10289000174908601648006814490988884203DD12
:1028A000124800881249086011480068002802DABE
:1028B00000200F4908601048006810490860074868
:1028C00000680D490860BDE8F0870000080000209E
:1028D0008C050020620000200000C8427C0500201A
:1028E000040E00200000C84300004842900500206C
:1028F0005C0500200000F0418005002084050020D8
:102900006C0500206405002068050020600500209B
:1029100078050020700500207405002010B500F037
:10292000F3FF0B4908800B48007828B90A48007863
:1029300010B9FFF7C7FE02E0002008490860074809
:10294000006881B24FF0804000F073FC10BD0000C1
:1029500008000020630000200C0000205C0500201F
:102960000A480B4908604FF07C500A4908604FF054
:102970007E50094908604FF07C50084908600848BB
:10298000084908600848094908607047000030415C
:1029900064050020680500206C05002070050020FB
:1029A0009A99193F740500200000C0407805002066
:1029B0007047000001460020034A506820F4404060
:1029C00008435060704700000010024029B1064AD9
:1029D000D2690243044BDA6104E0034AD2698243BC
:1029E000014BDA61704700000010024029B1064A2D
:1029F00092690243044B9A6104E0034A926982435C
:102A0000014B9A61704700000010024029B1064A4C
:102A1000D2680243044BDA6004E0034AD26882437E
:102A2000014BDA60704700000010024030B5002111
:102A30000022002400232D4D6D6805F00C0121B10A
:102A4000042905D0082923D105E0294D056022E09D
:102A5000274D05601FE0254D6D6805F47012234D6C
:102A60006D6805F48034022505EB92421CB9214DB6
:102A7000554305600BE01D4D6D6805F400351DB133
:102A80001C4D5543056002E0194D5543056002E0B9
:102A9000174D056000BF00BF144D6D6805F0F001D3
:102AA0000909154D6B5C0568DD4045600F4D6D688B
:102AB00005F4E061090A104D6B5C4568DD408560F6
:102AC0000A4D6D6805F46051C90A0B4D6B5C456891
:102AD000DD40C560054D6D6805F44041890B074D2B
:102AE0006B5CC568B5FBF3F5056130BD00100240B5
:102AF00000127A0000093D0024000020340000206C
:102B000010B5FFF79FF80024E2E0C4EBC40072495F
:102B100001EB8000007D30B1012822D0032848D08D
:102B200004287CD18EE0C4EBC4006B4901EB80002B
:102B3000807C01280DD10121C4EBC400664A02EB60
:102B4000800001750021C4EBC40002EB80004175D8
:102B500006E00021C4EBC4005F4A02EB800041752F
:102B6000B3E0C4EBC4005C4901EB8000807C012829
:102B700012D10321C4EBC400574A02EB8000017557
:102B8000C4EBC40002EB800041750021C4EBC4001B
:102B900002EB800041740BE00021C4EBC4004E4AFC
:102BA00002EB80000175C4EBC40002EB80004175AC
:102BB0008BE0C4EBC400484901EB8000807C012815
:102BC0000DD00021C4EBC400434A02EB8000017524
:102BD0000221C4EBC40002EB8000417531E0C4EB7C
:102BE000C4003D4901EB8000807C012822D1C4EB68
:102BF000C40001EB8000407C401CC1B2C4EBC400A7
:102C0000354A02EB800041741E2913DB0421C4EB1A
:102C1000C40002EB80000175C4EBC40000E053E087
:102C200002EB800041750021C4EBC40002EB800080
:102C3000417406E00021C4EBC400274A02EB800087
:102C4000417542E0C4EBC400234901EB8000807C65
:102C500001280DD00021C4EBC4001F4A02EB800004
:102C600001750221C4EBC40002EB800041752AE02B
:102C7000C4EBC400184901EB8000807C01281BD103
:102C8000C4EBC40001EB8000407C401CC1B2C4EB2B
:102C9000C400114A02EB800041741E290CDB0421A0
:102CA000C4EBC40002EB800041750021C4EBC400FA
:102CB00002EB8000417406E00021C4EBC400064A28
:102CC00002EB8000417500E000BF00BF601CC4B291
:102CD000012CFFF61AAF10BDE809002030B50346FD
:102CE0000C461546002207E0184600F008F824F8C4
:102CF00012009B1C501C82B2AA42F5DB30BD01467B
:102D0000088870472DE9F05F80468A461746B8F17B
:102D1000006F02D33348804501D3BDE8F09FFEF732
:102D20003DFEA8F1006B4FEA9B25CBF34809C9F59E
:102D30000074A74200DC3C464DE04FF0006101EB1F
:102D400085208A142849FFF7C9FF00260BE009EB0C
:102D50000600254931F810004FF6FF71884200D077
:102D600003E0701C86B2A642F1DB00BFA6421BDA6C
:102D70004FF0006101EB8520FEF7A6FD002608E07C
:102D80003AF8160006EB0901174A22F81100701CE8
:102D900086B2A642F4DB4FF0006101EB85208A1475
:102DA000114900F023F804E022465146404600F065
:102DB0001DF8A74200D10FE06D1C4FF000090AEB8F
:102DC000440AA044381B87B2B7F5007F02DD4FF4F8
:102DD000007400E03C46B0E700BFFEF7B5FD00BF61
:102DE0009BE7000000000108E80500202DE9F04104
:102DF00005460E461746002407E036F8141028460C
:102E0000FEF7ACFDAD1C601C84B2BC42F5DBBDE836
:102E1000F081704710B500F001F810BD0CB500202E
:102E2000019000903348006840F4803031490860D8
:102E300000BF3048006800F4003000900198401C4A
:102E40000190009818B90198B0F5A06FF1D1294808
:102E5000006800F4003010B10120009001E0002073
:102E600000900098012843D12348006840F01000EA
:102E7000214908600846006820F003000860084601
:102E8000006840F0020008601A484068194948602C
:102E90000846406848600846406840F480604860E2
:102EA0000846406820F47C1048600846406840F4BA
:102EB000E81048600846006840F08070086000BF75
:102EC0000C48006800F000700028F9D009484068FC
:102ED00020F00300074948600846406840F00200BF
:102EE000486000BF0348406800F00C000828F9D192
:102EF0000CBD00000010024000200240042808D150
:102F00004FF0E021096941F004014FF0E022116126
:102F100007E04FF0E021096921F004014FF0E022C1
:102F2000116170477047000010B51348006840F009
:102F300001001149086008464068104908400E49E0
:102F40004860084600680E4908400B49086008467A
:102F5000006820F4802008600846406820F4FE00E5
:102F600048604FF41F008860FFF754FF4FF0006087
:102F70000449086010BD0000001002400000FFF886
:102F8000FFFFF6FE08ED00E01CB50121194800F036
:102F9000E0F868B3FFF7B4FD002001901FE09DF852
:102FA0000400C0EBC000144901EB8000407D00909C
:102FB0009DF80000032804D1012010490880082052
:102FC00048809DF80000042804D101200B490880A6
:102FD0000A2048809DF80400401CC0B201909DF872
:102FE00004000128DBDB0121024800F0A3F800BF48
:102FF0001CBD000000040040E8090020580000202B
:103000007FB505460C4601210220FFF7DFFCADF835
:103010000850ADF804400020ADF80600ADF80A00F5
:10302000012211460D4800F0A5F801A90B4800F057
:1030300003F91D208DF8000000208DF80100032009
:103040008DF8020001208DF803006846FEF7A6FE09
:103050000121024800F071F87FBD0000000400402B
:103060007FB505460C4601210420FFF7AFFCADF803
:103070000850ADF804400020ADF80600ADF80A0095
:10308000012211460C4800F075F801A90A4800F029
:10309000D3F81E208DF8000000208DF801000120DB
:1030A0008DF802008DF803006846FEF777FE0121D7
:1030B000014800F042F87FBD0008004010B5012132
:1030C000174800F046F848B30121154800F032F8DF
:1030D00014480088401C13490880088800EBD07110
:1030E0004910A0EB410109B9FFF718FC0D48008811
:1030F000642813DB00200B4908800B480068401C43
:103100000949086009480068401C084908600848E7
:103110000068401C0649086001F000FD10BD000079
:1031200000080040A005002094050020980500201C
:103130009C050020CA430282704721B1028842F0F8
:103140000102028004E002884FF6FE731A400280FA
:10315000704730B50246002000230024158A05EA96
:103160000103958905EA010413B10CB1012000E0C7
:10317000002030BD1AB183890B43838102E083892B
:103180008B4383817047000070B500240022002328
:10319000058C4FF6FE7635400584028C8388048BBF
:1031A0004FF68F752C40B51E2C400D882C43751E94
:1031B0002A400D892A434D882A43144DA8420BD03A
:1031C000134DA84208D0134DA84205D0124DA84275
:1031D00002D0124DA84213D14FF6F7752A404D89FF
:1031E0002A434FF6FB752A408D882A434FF6FF6528
:1031F0002B404FF6FF552B408D892B43CD892B4318
:1032000083800483CD888586028470BD002C0140B4
:1032100000340140004001400044014000480140AA
:103220000A460021018B4FF6F773194011430183C1
:103230007047818670470000002202881D4B98422B
:103240000ED01D4B98420BD0B0F1804F08D01B4BD5
:10325000984205D01A4B984202D01A4B984204D19A
:103260004FF68F731A404B881A43174B984207D07A
:10327000164B984204D04FF6FF431A40CB881A43AE
:1032800002808B8883850B8803850A4B98420BD07C
:10329000094B984208D00E4B984205D00D4B9842EE
:1032A00002D00D4B984201D10B7A03860123838211
:1032B00070470000002C0140003401400004004031
:1032C00000080040000C00400010004000140040C6
:1032D00000400140004401400048014010B540F268
:1032E00025511D4800F04AF810B31B4800F002F9C0
:1032F000C4B21A48008800F40040C8B917480088D2
:1033000000F4804060B10A2C03D0002013490880EB
:1033100020E01248008840F400401049088019E07D
:103320000D2C06D10D48008840F480400B490880E0
:1033300010E00A480088C0F30D0009490C54074802
:103340000088401C0549088008460088C72801DD20
:103350000020088010BD000000380140AC050020AE
:10336000140E002021B1828942F40052828104E0CF
:1033700082894DF6FF731A408281704770B502460C
:10338000002400230025002040F66A16B14200D137
:1033900000BFC1F3421501F01F03012606FA03F333
:1033A000012D02D19689334006E0022D02D1168A02
:1033B000334001E0968A33400C12012606FA04F4E9
:1033C0001688344013B10CB1012000E0002070BD1C
:1033D000F0B50346002400260025002040F66A17B9
:1033E000B94200D100BF1846C1F3421401F01F06D4
:1033F000012707FA06F5012C01D10C3004E0022C5C
:1034000001D1103000E014301AB107682F43076073
:1034100002E00768AF430760F0BD00002DE9F04708
:1034200086B005460E460024A24600BFA1460027EE
:10343000B08900B100BF2F462C8A4CF6FF700440C3
:10344000F08804432C82AC894EF6F3100440B08817
:1034500031890843718908430443AC81AC8A4FF633
:10346000FF400440B0890443AC8201A8FFF7DEFAB4
:103470001F48874202D1DDF810A001E0DDF80CA062
:10348000A88900F4004040B10AEBCA0000EB0A1022
:1034900031684900B0FBF1F807E00AEBCA0000EB25
:1034A0000A1031688900B0FBF1F86420B8FBF0F035
:1034B00004012009642101FB1089A88900F400405F
:1034C00040B1322000EBC900B0FBF1F000F0070082
:1034D000044308E0322000EB09106421B0FBF1F056
:1034E00000F00F0004432C8106B0BDE8F087000017
:1034F0000038014001468888C0F30800704700BFCB
:10350000FEE7490050EAC12018BF04204A0D18BF49
:1035100040F0010040F2FF72B2EB515F08BF40F093
:103520000200012808BF052070472DE9F0414F1E19
:1035300000EBC7010446D1E9000115461E4637F0ED
:1035400006020DD02A46334601F04AFE7F1E04EBE8
:10355000C703D3E9002301F08DFB37F00602F1D158
:10356000022F25D0042F13D0062F18BFBDE8F081FD
:103570002A46334601F034FED4E90A2301F07AFBEF
:103580002A46334601F02CFED4E9082301F072FBF1
:103590002A46334601F024FED4E9062301F06AFBF3
:1035A0002A46334601F01CFED4E9042301F062FBF5
:1035B0002A46334601F014FED4E9022301F05AFBF7
:1035C0002A46334601F00CFED4E90023BDE8F04161
:1035D00001F050BB002213461046014901F006BC21
:1035E0000000F03F012202F098BB00221346104673
:1035F000114601F0FBBB30380A2801D20120704788
:103600000020704700BF704710B50748807B48B165
:103610000120064908600A2000F02EF80020044925
:10362000C1F8A40110BD0000040E0020A4812142B5
:103630000080214210B56FF00400FFF75FFC0A48DC
:1036400000680A49B0FBF1F00949087008460078A3
:1036500000EB4001C1EBC0104FF6FF7101EAC00062
:103660000449088010BD00001000002000127A00FC
:1036700054000020560000200146114A12884A4397
:103680004FF0E0235A6100229A611A46126942F013
:1036900001021A6100BF4FF0E022106900F0010240
:1036A0001AB100F48032002AF5D04FF0E0221269FE
:1036B00022F001024FF0E0231A6100229A61704764
:1036C000560000200146114A12784A434FF0E02389
:1036D0005A6100229A611A46126942F001021A6187
:1036E00000BF4FF0E022106900F001021AB100F4AF
:1036F0008032002AF5D04FF0E022126922F0010258
:103700004FF0E0231A6100229A61704754000020B4
:103710001FB501210820FFF769F90920ADF80C0059
:1037200004208DF80F0003208DF80E0003A9144823
:10373000FEF774F901210846FFF758F9002101202E
:10374000FEF74CF90120019000208DF808000820B8
:103750008DF8090001208DF80A0001A8FEF76AF82B
:1037600006208DF8000002208DF8010001208DF860
:1037700002008DF803006846FEF710FB1FBD000035
:10378000000C014070B50646002500240948006879
:103790000A21B0FBF1F43C20B4FBF0F5C5EB0510B9
:1037A000A4EB800423462A4603A13046FCF73EFDE5
:1037B00070BD000094050020253033643A25303276
:1037C000640000002DE9F04F8DB000200C900B90AC
:1037D0000A900C210620FEF71DFA3449088008469D
:1037E000008802F0A1F8064631480168304602F030
:1037F000E0F904462D48008802F096F806462D4868
:103800000168304602F0D8F80546214601F076FFFF
:103810000C90294801680C9801F070FF019001F0AC
:10382000D3FE804600F0BAFA06460F4623480068E9
:1038300001F0CAFE32463B46CDE9020101F0D0FC60
:10384000CDE906011E48006801F0BEFECDE9040185
:10385000DDE9062301F00EFA04460D46174801681B
:103860001748006802F0A8F8064601F0ADFE2246AF
:103870002B46CDE9080101F0B9FA824601F0C8F9FA
:103880000B900B9801F0A0FE06464FF066320D4BF0
:1038900001F0B0FD044601F0BBF90A900A9802F06D
:1038A0000BF880B20DB0BDE8F08F00005000002092
:1038B0003800002044000020480000204000002084
:1038C0003C0000206612714010B500214FF080408E
:1038D000FFF7AFFC4FF4FA70FFF7F4FE0420FEF799
:1038E0007FF9044640F6DC70844201DA0448048023
:1038F0000448006881B24FF08040FFF79AFC10BD89
:10390000520000205C0500202DE9F8430025002628
:10391000FFF7DAFF4148008840F21631884214DA96
:103920003E48008802F000F880463D4800233D4AAA
:1039300019460090404600F037FD074601F0BCFFF5
:1039400039490988084486B249E03448008840F281
:103950008661884214DA3148008801F0E5FF80462C
:1039600032482F4B324A2F490090404600F01CFD50
:10397000074601F0A1FF2C490988084486B22EE0D1
:103980002648008840F65431884214DA23480088DB
:1039900001F0CAFF80462748244B274A244900905B
:1039A000404600F001FD074601F086FF1E490988E8
:1039B000084486B213E01948008801F0B5FF80463C
:1039C0001E481C4B1E4A1C490090404600F0ECFC6F
:1039D000074601F071FF14490988084486B20024A3
:1039E0000CE01849601C31F8100021F81400601C2C
:1039F00031F81000284485B2601CC4B2072CF0DBFB
:103A00001048C681C089284485B22846E91705EBCD
:103A10005171CE103046BDE8F883000052000020FE
:103A20000000C842008045440400002000004843D4
:103A300000C0D04400009643004035450000D2430A
:103A400000A07F45BA0500202DE9F0470A21022099
:103A5000FEF7E0F8824601F074FB06464FF066324E
:103A6000074B01F0BDFB04460022064B01F0BEF9F6
:103A7000804601F0CDF804490860BDE8F0870000F9
:103A80006626424000FEAF40000000202DE9F041D4
:103A90008AB0A5A000680990A4A00068089002A8B8
:103AA000FFF770FE0020102302AA01460090FEF7E7
:103AB000FBFC9F48006801F087FD064600229D4BF5
:103AC00001F052FB0BD29A48006801F07DFD0646DA
:103AD00032460B4698A105A8FCF7A8FB0AE09448DB
:103AE000006801F071FD064632460B4694A105A818
:103AF000FCF79CFB0120102305AA00210090342034
:103B0000FEF7D2FC9048D0F8012090A107A8FCF75E
:103B10008DFB0020102307AA014600905820FEF7D5
:103B2000C3FC002010210B46894ACDE90010014654
:103B30007020FEF7C9F901200F237F22194600905B
:103B40000020FEF749FA8348007800286BD17E49AF
:103B5000D1F80110804A128891420BD17E49098820
:103B60007E4A1288881A002801DB014600E04142A3
:103B70000A2903DD79480088774908807249D1F81D
:103B80000110754A1288501A002801DB014600E036
:103B90004142012904DC6C48D0F801006E490880DC
:103BA0006D480088642190FBF1F084B26A48008877
:103BB00090FBF1F201FB12000A2190FBF1F085B2BB
:103BC0006548008890FBF1F201FB12001FFA80F8B3
:103BD00004EB44004006020E012311210020FEF7F1
:103BE000B9F905EB45004006020E01231121192009
:103BF000FEF7B0F908EB48004006020E0123112140
:103C00003220FEF7A7F95648006864214843FF2197
:103C100090FBF1F6102003233246302100904E2015
:103C2000FEF7F8FB27E0012010234EA2112100909F
:103C30000020FEF739FC012010234AA22121009028
:103C40000020FEF731FC0120102349A23021009012
:103C50000020FEF729FC0120032309AA1621009069
:103C60000C20FEF7BDFB0120022308AA28210090AA
:103C70001520FEF7B5FB1020022300904048028873
:103C800018214E20FEF7C6FB012010210B46304ABA
:103C9000CDE9001018215E20FEF716F939480078AA
:103CA00018B92C480078012812D101200F211023C7
:103CB000354ACDE9001018217020FEF705F90120E2
:103CC000102332A2302100906820FEF7EDFB27E0A0
:103CD0002F48007890B101200F2110232A4ACDE906
:103CE000001018217020FEF7EFF80120102329A200
:103CF000302100906820FEF7D7FB11E001200F2152
:103D00001023254ACDE9001018217020FEF7DCF8B9
:103D1000012010231FA2302100906820FEF7C4FB71
:103D20000AB0BDE8F08100002A2B2C002D2E0000E7
:103D3000000000200000244025312E3266000000E3
:103D400025322E3166000000040E0020256400009C
:103D50009E0000200C0000206000002008000020D1
:103D60005C05002020202020202020202020000092
:103D700020202020202020202020202020000000A3
:103D80000400002063000020DA0000204F464600B7
:103D900062000020204F4E00BE0000202DE9F04DB3
:103DA000C84A002490B0914205DA21F000439342C2
:103DB00001D805D120B110B0BDE8F04DFFF712BC1D
:103DC000B1F5801F1BDA53EA000209D0002911DA8D
:103DD0000120FCF748FB10B0BDE8F04DFFF705BC33
:103DE0000220FCF740FBFFF7F5FB10B081F000412B
:103DF000BDE8F08D6FF03504362201F08EFF04EB44
:103E00002152C1F31308B049A2F2FF33414401F437
:103E1000801282F07F6103EB225281F040510092C8
:103E200041EA08010022A94B01F0E4FA044608F136
:103E30000200A74EC0F313000D467E44032867D24C
:103E4000D6E90023204601F029F91ED10098002868
:103E500002BFD6E9000110B0BDE8F08D01F05AF9BB
:103E600007460C469B4A9C4B01F0BAF906460D46A4
:103E70009A4A9B4B3846214601F0B2F910B03246BF
:103E80002B46BDE8F04D00F0F5BE4FF05532954B96
:103E90002046294601F0A4F90022934B01F09EFA36
:103EA00006460F4622462B461046194601F098F961
:103EB00032463B4601F094F9064600980F46F0B1B1
:103EC00001F028F980468A46824A834B01F088F93E
:103ED00032463B4601F082FA22462B4601F08AFA2E
:103EE00005460C467D4A7E4B4046514601F078F926
:103EF00010B02A462346BDE8F04D01F07BBA0B46D0
:103F000010B0324620462946BDE8F04D01F072BAA5
:103F100000224FF08043204600F0ACFE02460B46E4
:103F20002046294600F062FF06460F46009801F041
:103F3000F1F8CDE9040132463B461046394601F01E
:103F40004FF90C9069480C9A4044019009910B4636
:103F5000104601F045F98246024665488B46C8F195
:103F600051080B4608F5D72803217844FFF7DDFAFE
:103F700052465B4601F034F90A905E480D91524674
:103F80005B4604217844FFF7D0FA099B0C9A01F0B4
:103F900027F9844601980D9B40EA080860460A9A72
:103FA00000F068FE83460891B8F1000F4EDD4FF037
:103FB000FF322046294601F0B0FE22462B4601F092
:103FC0000FF9804600988A4660B3DDE90401414A52
:103FD000414B01F005F9099100905A46404651467F
:103FE000089B00F047FE32463B4601F0F9F8099B7A
:103FF000009A00F03FFE4246534601F0EFF9224698
:104000002B4601F0F7F904460D46DDE90401334A79
:10401000334B01F0E5F810B022462B46BDE8F04DD9
:1040200001F0E8B95A464046089B00F023FE3246AC
:104030003B4601F0D5F84246534601F0CFF910B0A7
:1040400022462B46BDE8F04D01F0C8B9009840B3B8
:10405000DDE904011F4A204B01F0C2F880468A4680
:104060005A4620462946089B01F0C4F932463B4691
:1040700001F0B6F84246534601F0BCF922462B4601
:1040800001F0B8F904460D46DDE90401134A144B6A
:1040900001F0A6F810B022462B46BDE8F04D01F025
:1040A000A9B90B465A462046294601F0A3F93246E3
:1040B0003B4601F095F810B022462B46BDE8F04D86
:1040C00001F08CB90000F07F645F09000000F03F50
:1040D000D2380000763C7935EF39EA3D0000E0FE49
:1040E000422EE63F5555D53F0000E03F86EBF9FFF5
:1040F0006A370000683700001CB5FDF723FEFFF7A4
:1041000099FA4FF4A060FDF781FE4FF4E13000F022
:1041100019FD472144F61F60FEF772FFFDF7CAFA4A
:10412000FDF75EFAFDF7C4FDFDF774FF00F0DAFC61
:10413000FEF716FC40F2CF216320FEF791FFFDF75A
:104140006FFE012040218023834ACDE90010002129
:104150000846FDF7B9FEFEF70DF84FF47A70FFF749
:104160008BFAFFF751FAFFF72DFB7C4908800846D0
:1041700000887B49088000207A4908700BE0784865
:1041800000887949774A127821F81200754800783A
:10419000401C74490870734800780828EFDB002041
:1041A0003F237F2201460090FDF716FFD2E06F48C3
:1041B0000088642190FBF1F201FB1200002855D128
:1041C000FFF700FB65490880FFF73EFC6348008865
:1041D000322804DB664800886049088003E05F48B5
:1041E000008863490880002500240CE06149601CB8
:1041F00031F8100021F81400601C31F81000284438
:1042000085B2601CC4B20E2CF0DB544800885949BA
:1042100088830846808B284485B20F2095FBF0F0F8
:104220004E49088008460088052808DB08460088B3
:10423000322804DC00205049087050490870474873
:104240000088052803DB45480088322807DD4B48F5
:10425000007820B948480078401C47490870464813
:104260000078082802DB012044490870444800789F
:1042700060B93E4800884FF4487190FBF1F201FBB1
:10428000120018B9FFF702FCFDF774FF3D480088E3
:1042900080B300F0ADF8FFF7B7F93A484088082836
:1042A00010D13748007868B93748007838B1002015
:1042B00035490870354908603549086002E0012039
:1042C000314908703348007820B100203149087026
:1042D0002F4908602A4800782F4908700020294992
:1042E0000880FEF74DF92D48006882B22C492D4810
:1042F000FEF708FD2A48D0F8050000280EDD284802
:10430000D0F80500C0EB001000EB80001F490968E1
:10431000B1EBC00F02D901201B4908702048D0F82A
:10432000090000280EDD1E48D0F80900C0EB00107F
:1043300000EB800016490968B1EBC00F02D90120DB
:104340001449087009480088401C08490880642006
:10435000FFF7B8F92BE7000055010020040000200A
:10436000080000200E000020BA0500200A000020EE
:1043700006000020CA0500200D0000200C000020CF
:1043800064000020580000206200002098050020F2
:104390009C0500206300002065000020A40500208B
:1043A000040E002004FC00082DE9FC5F06460F46C1
:1043B00014461D46DDF830803946204601F004FCE5
:1043C00029460190404601F0FFFB834639463046BE
:1043D00001F0FAFB5946009001F0EEFA824601998D
:1043E00001F08CF98146294601F01AF9BDE8FC9FDD
:1043F00064484088062843D163480078072823D0C2
:1044000005DC48B105280FD0062838D114E008286B
:1044100023D00D2833D129E05C48D0F80100401D9D
:104420005A49C1F801002AE05848D0F80500401C5C
:104430005649C1F8050022E05448D0F80900401C54
:104440005249C1F809001AE05048407B08B90120E0
:1044500000E000204D49487311E04C48807B08B9CA
:10446000012000E000204949887308E04748C07BEC
:1044700008B9012000E000204449C87300BF47E0AC
:1044800040484088072843D13F480078072823D078
:1044900005DC48B105280FD0062838D114E00828DB
:1044A00023D00D2833D129E03848D0F80100401F2F
:1044B0003649C1F801002AE03448D0F80500401E12
:1044C0003249C1F8050022E03048D0F80900401E0A
:1044D0002E49C1F809001AE02C48407B08B9012098
:1044E00000E000202949487311E02848807B08B982
:1044F000012000E000202549887308E02348C07BA4
:1045000008B9012000E000202049C87300BF00BFA7
:104510001E48D0F80100B0F5C87F04DD4FF4C87024
:104520001A49C1F801001948D0F80100962803DAA9
:1045300096201649C1F801001448D0F805003C281F
:1045400003DD3C201149C1F805001048D0F80500F2
:10455000002803DA00200D49C1F805000B48D0F807
:1045600009003C2803DD3C200849C1F80900074840
:10457000D0F80900002803DA00200449C1F8090036
:10458000704700005800002064000020040E002046
:1045900010B58AB004464EA0006807904DA0006890
:1045A00006904DA0006805904CA00068039020780C
:1045B00010234BA2002100900846FDF775FF2078DC
:1045C000042307AA002100901020FDF709FF4548A9
:1045D000D0F8052044A108A8FBF728FE2079102375
:1045E00008AA002100905820FDF75EFF6078102394
:1045F0003FA2194600900020FDF756FF6078042383
:1046000006AA102100900846FDF7EAFE3548D0F8CA
:10461000092035A108A8FBF709FE6079102308AA34
:10462000194600905820FDF73FFFA078102331A2D3
:10463000202100900020FDF737FFA078042305AA71
:10464000202100901020FDF7CBFE2648407B30B1A2
:104650000A208DF810000B208DF8110005E00C20C9
:104660008DF810000D208DF81100A079022304AA06
:10467000202100905820FDF7B3FEE07810231EA201
:10468000302100900020FDF70FFFE078032303AAFC
:10469000302100901020FDF7A3FE1248807B50B11E
:1046A000E0790E211023154ACDE90010322158205F
:1046B000FDF70AFC09E0E0790E211023104ACDE94C
:1046C000001032215820FDF7FFFB0AB010BD00009A
:1046D0000001020304050203060708090E0F10007B
:1046E000312E0000040E0020252D32646D696E000D
:1046F000322E0000332E0000342E00006600002011
:104700008200002010B588B0044633A000680790EE
:1047100032A00068069032A103C9CDE9040132A09D
:10472000006803902078102330A2002100900846F2
:10473000FDF7BAFE2078042303AA00210090102080
:10474000FDF74EFE2A48C07B50B120790E21102380
:10475000284ACDE9001000215820FDF7B5FB09E0FB
:1047600020790E211023244ACDE900100021582081
:10477000FDF7AAFB6078102320A2194600900020C4
:10478000FDF792FE6078062304AA102100900846E7
:10479000FDF726FEA078102319A22021009000200A
:1047A000FDF782FEA078042306AA202100901020A5
:1047B000FDF716FEE078102312A2302100900020B1
:1047C000FDF772FEE078022307AA30210090102046
:1047D000FDF706FE08B010BD1F2000001B1C1D1EAB
:1047E0001718191A1314000011121314352E000093
:1047F000040E0020FA00002016010020362E0000D2
:10480000372E0000382E00001CB504A103C9CDE9E5
:1048100000016846FFF7BCFE1CBD0000010101005D
:10482000010101011CB504A103C9CDE900016846DD
:10483000FFF7AEFE1CBD00000101010001010100F7
:104840001CB504A103C9CDE900016846FFF7A0FE2D
:104850001CBD000001000101010101011CB504A102
:1048600003C9CDE900016846FFF792FE1CBD0000B8
:1048700001000101010001011CB504A103C9CDE93A
:1048800000016846FFF73EFF1CBD0000010100016A
:104890000100000000B585B032A00068049032A08D
:1048A0000068039031A00068029031A00068019078
:1048B00000203F237F2201460090FDF78DFB012061
:1048C000022302AA002100900846FDF789FD01207D
:1048D000102328A2002100902020FDF7E5FD0120F3
:1048E000022301AA002100903020FDF779FD01206C
:1048F000022303AA102100900020FDF771FD012082
:1049000010231DA2194600902020FDF7CDFD0120A7
:10491000022304AA202100900020FDF761FD012060
:10492000102319A2202100900846FDF7BDFD0120AB
:10493000102317A2302100900020FDF7B5FD0120C3
:1049400010232722302100901846FDF7D7FC0120C4
:10495000102310A2302100902020FDF7A5FD05B006
:1049600000BD0000252600002324000021220000B5
:10497000282900003A2000003A20323032312E300F
:10498000352E3034000000003A2056312E3600001B
:10499000515100003A20313039313939363633340B
:1049A000000000001CB504A103C9CDE90001684660
:1049B000FFF7EEFD1CBD0000010100010101010136
:1049C0001CB504A103C9CDE900016846FFF7E0FD6D
:1049D0001CBD000001010001010100011CB504A182
:1049E00003C9CDE900016846FFF78CFE1CBD00003D
:1049F00001000101010000001CB501200E2110235F
:104A0000044ACDE9001012217220FDF75DFA00F092
:104A100055F81CBD660000201CB504A103C9CDE9F2
:104A200000016846FFF76EFE1CBD00000101010099
:104A3000010000001CB504A103C9CDE900016846CE
:104A4000FFF7A6FD1CBD00000001010101010101ED
:104A50001CB504A103C9CDE900016846FFF798FD24
:104A60001CBD000000010101000101011CB504A1F1
:104A700003C9CDE900016846FFF744FE1CBD0000F4
:104A800000010101010000001CB504A103C9CDE92A
:104A900000016846FFF736FE1CBD00000001010161
:104AA0000000000010B50246012000E050430B1E3C
:104AB000A1F10104E1B2F9D110BD000011200849B3
:104AC00008704FF48C70C1F801000520C1F8050092
:104AD0001420C1F80900012048738873C873704717
:104AE000040E002010B50A48006882B209490A483D
:104AF000FEF7F4F807480078112808D0FFF7DEFF2A
:104B00000348006882B203490348FEF7FBF810BD72
:104B1000A4050020040E002004FC000805490968D3
:104B200088B230B90021044A1170044A1160044A65
:104B3000116070472001214262000020980500208A
:104B40009C05002010B586B00446012144F2040003
:104B5000FDF74CFF4FF40070ADF8140003208DF802
:104B6000160018208DF8170005A91C48FCF756FF01
:104B70004FF48060ADF8140004208DF8170005A9EB
:104B80001648FCF74BFF25208DF8000003208DF818
:104B900001008DF8020001208DF803006846FDF742
:104BA000FDF801940020ADF80800ADF80A00ADF85A
:104BB0000C00ADF810000C20ADF80E0001A908485B
:104BC000FEF72CFC012240F225510548FEF700FCBF
:104BD00001210348FEF7C6FB06B010BD00080140E6
:104BE0000038014010B500290AD00878002807D005
:104BF00005487844FBF7F6FF002801D0002010BDDF
:104C00000248784410BD0000DA2B0000D22B0000CF
:104C100021F00042A2F16052B2F5801F01F0004382
:104C200028BFD2F17F6C0BD95FEA001C43EAC202B5
:104C300042EB507018BF704728BF20F0010070474A
:104C4000B2F5801FBCBF184670474FEA410C1CF5F7
:104C5000001F02D2084600F076BF70B500F06AFB74
:104C600000000089FFF7F6BF4FF00040A0F580007C
:104C70007047000010B591EA030F48BF83F000436E
:104C800000F1C083841A71EB030C05D2121943EBB7
:104C90000C03001B61EB0C01DFF824E14FEA115417
:104CA000A4EB135C1EEA430F18BF9EEA445F73D067
:104CB00023EA0E03DCF1200E21EA045143F48013B1
:104CC00032D322FA0CFE10EB0E0023FA0CFE41EB5D
:104CD0000E01CCF1200E03FA0EFE10EB0E0051F186
:104CE0000001B1F5801FCCF1200E32D201EB04514E
:104CF00012FA0EF2BDE8104058BF7047401C38BF92
:104D00005FEA420218BF7047002814BF20F001007C
:104D100041F100014FEA410313F5001F38BF70470E
:104D2000A1F1C04100F054BB012A43EB0302ACF1F6
:104D3000200CDCF11F0E32BF4FF0000E23FA0CF3F3
:104D400010EB030041EB0451B4EB115FD0D0A1EBA9
:104D5000045101F5801149085FEA300001EB04516C
:104D60000ED350F1000038BF12FA0EFE08D1BDE894
:104D70001040C9E7401C38BF5FEA4202CAD1C3E70E
:104D8000BDE810404FEA410313F5001F38BF7047DC
:104D9000A1F1C04100F01CBB9EEA445F08D011EABB
:104DA0005E0FBDE8104004BF01F0004100207047D5
:104DB000BDE8104070B500F0BDFA00BF64FBBE3E18
:104DC0000000E0FF02494FF0000000F074BF00BF98
:104DD0000000F87F491058BFC1F140415B1058BF37
:104DE000C3F140438B42EFF3008070472DE9C0418F
:104DF00030B4DFF8A0C23CEA111418BF3CEA131427
:104E000000F0EC8081EA03051CEA111444EAD57431
:104E100018BF1CEA131500F0C780A4EB05044FF07F
:104E2000004545EAC12145EAC32341EA505143EA1E
:104E3000525304F17F74994204F500344FEAC020C4
:104E40004FEAC22208BF904200F09C804FEA1365EF
:104E50000FF24016765D4FEA134506FB05F7C7F1E2
:104E6000807706FB07F74FEAD737A7FB0368764240
:104E7000C8F58038A7FB06CE38BFA8F1010807FBAC
:104E800008E64FF0000EA6FB028CE6FB03CEDCF139
:104E9000000CCEF1004E38BFAEF1010EA6FB0C584F
:104EA0004FF000074FF00005E6FB0E87A1FB08C698
:104EB000A0FB07CE16EB0E0645F10005E1FB0765EA
:104EC00015F1E04E7EBFA4F580345FEA46066D41E1
:104ED00016F1800745F100054FEA17274FEA0666ED
:104EE00047EA0567A6F1DE46B6F1805F4FEA152571
:104EF0001FD9384624F0010C05EBC471BCF1FE6FDC
:104F000001EB0C1102D8F0BCBDE8008124425CBF6B
:104F100001F5801E9EEAC47F02D4F0BCBDE800818A
:104F2000244238D4F0BCA1F1C041BDE8004100F0FA
:104F30004FBA4FEAD22242EA43524FEAD323A7FBA9
:104F400002864FEAD02040EA415007FB03661EEA82
:104F50000E0F4FEAD12105FB026658BFA6EB0056A3
:104F6000B6EB00564FEA520E4EEAC37E18EB0E0E19
:104F700056EB530EBDD518EB02085E417F1C55F170
:104F80000005B6E74FF480154FF000074FF000061C
:104F90004FF00008ADE7F0BC4FF0000001F1C04158
:104FA00001F00041BDE8008111EA0C1F0CEA131565
:104FB00000D00CE013EA0C1F00F025804FF0000039
:104FC000F0BC81EA030101F00041BDE80081F0BCC2
:104FD000BDE8004181EA030100F0FAB9F0BCBDE888
:104FE000004170B500F0A6F9097EFC3E00F007B85C
:104FF00081EA03014FF0000001F00041704781EAAF
:10500000030100F0E5B9F0BCBDE800414FF000003D
:1050100021497047FFFDFBF9F7F5F4F2F0EEEDEBF7
:10502000E9E8E6E4E3E1E0DEDDDBDAD8D7D5D4D3A6
:10503000D1D0CFCDCCCBCAC8C7C6C5C4C2C1C0BFF2
:10504000BEBDBCBBBAB9B8B7B6B5B4B3B2B1B0AFF8
:10505000AEADACABAAA9A8A8A7A6A5A4A3A3A2A1DC
:10506000A09F9F9E9D9C9C9B9A9999989797969597
:1050700095949393929191908F8F8E8E8D8C8C8B33
:105080008B8A8989888887878685858484838382BB
:10509000828181800000FF070000F87F51EA030C45
:1050A00017D41CF5801F58BFBCF5801F00F1068087
:1050B000994218BF704708BF9042704707D711F553
:1050C000801F58BF13F5801F19D499427047894239
:1050D00070471CF5801F08D5BCF5801FF7D58B42A3
:1050E00018BF704708BF824270474FF4001C1CEB8A
:1050F000410F38BF1CEB430F01D28B42704770B594
:1051000000F018F9922449004FF000514FF08053FD
:10511000FFF760BE10F0004248BF4042B0FA80F393
:1051200010FA03F10AD0C3F11D0303F580634FEABF
:10513000415002EB035202EBD12170474FF00000C7
:105140007047B0FA80F310FA03F10AD0C3F11D03DF
:1051500003F580634FEA41504FEA035202EBD1213D
:1051600070474FF00000704751EA030C17D41CF54C
:10517000801F58BFBCF5801F00F10680994218BF00
:10518000704708BF9042704707D711F5801F58BF7E
:1051900013F5801F19D499427047894270471CF556
:1051A000801F08D5BCF5801FF7D58B4218BF70470C
:1051B00008BF824270474FF4001C1CEB410F38BF00
:1051C0001CEB430F01D28B42704770B500F0B2F870
:1051D000922449004FF000514FF08053FFF7FABD81
:1051E000DFF848C170B51CEA111E1EBF1CEA13157A
:1051F0009EEA0C0F95EA0C0F00F06F8081EA030421
:1052000023EA4C134EEAD47E21EA4C1141F480117A
:1052100043F48013AE44A1FB024CA0FB0365AEF146
:105220007F7E361955EB0C05A1FB034C4CF10003B6
:10523000A0FB021C16EB0C06654153F1000309426A
:1052400018BF46F0010613F4007F0BD14FEA03317B
:105250004FEA0530340341EA155140EA16506FF029
:1052600003020AE04FEAC3214FEAC520F40241EAF3
:10527000555140EA56506FF0020202EB2E4201EB0C
:10528000025585EACE710AD05FEA440C18BF24F0BB
:10529000004450F1000041F1000120EAD47040F2D6
:1052A000FE7C624500D270BDA84214BF4FF080441E
:1052B0004FF04044002E08BF0024BEF1806FA8BF0D
:1052C000A1F1C041BDE8704080F282804FF0000043
:1052D00001F1C04101F0004170479EEA0C0F0CEA59
:1052E000131518BF95EA0C0F06D04FF0000081EAA5
:1052F000030E0EF0004170BD00F01CF88900013E65
:1053000000F007B800F009B84FEA430C5FEA5C5CB4
:1053100008D081EA030100F05BB84FEA410C5FEA74
:105320005C5CF6D14FF00000014970470000FF07B8
:105330000000F87F0EF1020E2EF0030E5EF8046BF3
:10534000364205D4012A43EB030515F5001F12D898
:10535000012841EB010C1CF5001F0CD80ED14FEABF
:10536000D17C15F5001F0CEB4C0C0CF1020C08BFA6
:105370004CEBD37C04E04FF0080C01E04FEAD37C07
:105380000CEB4C0526FA05F606F00706B6F1040C00
:1053900006D20EEB860CBDE870404CF0010C604765
:1053A000DFE80CF0090B02024FF000414FF0000063
:1053B000A1F5002170BD19461046012851EB0104EA
:1053C00018BFD4F5001484BF002001F0004170BD67
:1053D0000808A0F500114FEA3101704791EA030F68
:1053E00010B581F000413FF54DAC83F0004300F073
:1053F00009B8000010B591EA030F48BF83F00043DD
:105400003FF540AC841A71EB030C07D212198CF0F3
:10541000004C43EB0C03001B61EB0C01DFF8A4E133
:105420004FEA1154A4EB135C1EEA430F18BF9EEA27
:10543000445F00F0B08023EA6E03524221EA045137
:10544000C3EB6E0338BF5B1EDCF1200E25D322FABE
:105450000CFE10EB0E0043FA0CFE41EB0E01CCF1FA
:10546000200E03FA0EFE10EB0E0051F10001CCF1FC
:10547000200E29D412FA0EF201EB0451BDE81040BF
:1054800058BF7047401C1CBFB2F1004F7047002846
:105490000CBF491C20F00100704712EB020E43EBD9
:1054A000030218BF4FF0010E4EEA4202ACF1200C8D
:1054B000DCF11E0E54D943FA0CFE10EB0E0051F134
:1054C000FF31CCF11E0ED5D50EF1010E12FA0EFEF3
:1054D000404141EB010101EB445C5FEA5C5C10D9A7
:1054E00010EBDE7001EB045138BFBEF1004FBDE898
:1054F000104018BF704700280CBF491C20F0010065
:10550000704730D24FEAD42C11F5001124F4006416
:105510001BD0B1FA81F20B3AA41AA41ED2F12003D7
:10552000914030FA03F31943904001EBCC71002C09
:1055300001EB0451BDE81040A8BF704701F1C04124
:105540004FF0000001F000417047B0FA80F310FA0C
:1055500003F100D110BDE41A173C4805C90AE4E77D
:1055600001EB045110BD491001EB0451BDE810409E
:105570004FEA300002E04FF0000170474A0008BFD8
:105580000042F8D0B2F5001F28BF704701F000417B
:105590004FF0000070479EEA445F07D011EA5E0FAB
:1055A000BDE8104004BF002100207047BDE8104056
:1055B00070B5FFF7BFFE00BF40DFF63E83F000414D
:1055C000104670470000E0FF43004FEAD30C4FEA5B
:1055D0003C0C43401FBF40070CF1605113F0FE4FDD
:1055E00070471CF0006F03D100200CF000417047A1
:1055F0000CF0004343EA507010B540EACC0000F0D4
:105600005CFA00BF000000924FEA0001FFF7E0BE25
:105610004FF000414FF00000A1F50021704700005D
:1056200090EA010F48BF81F0004100F1D482421A94
:105630003CBF801A89184FEAD0524FF07F4C1CEAC9
:10564000410FA2EBD15318BF9CEA026F00F03B80E0
:105650004FF0004C4CEA00204CEA012121FA03FCF7
:1056600010EB0C0C1ED202F1FF325FEA1C2040EB63
:10567000C25038BF70471CF07F0F4FEA400C18BF74
:10568000BCF17F4F38BF7047C3F12003994008BF7A
:1056900020F00100BCF17F4F38BF7047A0F1C0403F
:1056A00000F051BA4FEA3C00000A40EBC25028BF5C
:1056B0001CF0FF0F4FEA400CE6D018BFBCF17F4F43
:1056C00038BF7047EAE79CEA026F05D010EA5C0F2A
:1056D00008BF00F00040704710B500F0EEF900BFC1
:1056E00064FBBE3E401058BFC0F14040491058BF57
:1056F000C1F140418142EFF3008070474FF47F0CCD
:105700001CEAD0121EBF1CEAD11392EA0C0F93EAD6
:105710000C0F00F0858090EA010F48BF42F48072C0
:1057200040F4000C41F400002CF07F4120F07F4059
:1057300000B58142A2EB03020FF2081CACEB504E05
:10574000C0F100009EF800E04FEA4E0E00FB0EFC98
:1057500038BF49004FEA2C1C02F5FA020CFB0EF38D
:105760004FEACE1E4FEA112C4FEAC1210EEB635EC9
:1057700042EB22420EFB0CFC4FEA1C5300FB0311D0
:105780004FEA112C4FEA01310EFB0CFC4FEADC4CC6
:1057900000FB0C11C14228BF09184CEB03335DF824
:1057A00004EB10EB410143EBC250B2F57C0F38BF64
:1057B000704729D512F0F00F1CBF00F1C04000F077
:1057C00000407047008182838485868788898B8C1E
:1057D0008D8E8F919293959697999A9C9D9FA0A25A
:1057E000A3A5A7A8AAACAEB0B2B3B5B7B9BCBEC0AA
:1057F000C2C5C7C9CCCED1D4D7D9DCDFE2E6E9EC4B
:10580000F0F3F7FAFE0000004FEA400C0CF1807C48
:10581000BCF17E4F28BF7047B0F1C04000F093B993
:1058200090EA010F0CEAD11348BF42F4807262453E
:1058300038BF634507D213F47F0F16D080EA01000A
:1058400000F00040704710B500F037F9097EFC3ECB
:1058500000F005B880EA010000F00040704780EADF
:10586000010000F0004000F06EB912F47F0F04BF99
:105870000248704780EA010000F065B90000C07F6F
:1058800041000B0ED3F19E0208D950F400034FEAF9
:10589000032323FA02F048BF4042704710B500F0DE
:1058A0000CF900BF49922480002070476FF000423D
:1058B00082EA200070470000C10DD1F19E0206DB94
:1058C0004FEA002343F0004323FA02F070470042FE
:1058D00007D54FEA4001B1F1FE4F02D24FF0000070
:1058E000704710B500F0E9F8499224800020704715
:1058F0006FEA20007047000010F0004148BF4042AE
:10590000B0FA80F310FA03F2C3F19D030BD051EA11
:10591000C35101EB1220530638BF704700F101005C
:1059200008BF20F001007047B0FA80F310FA03F2CC
:10593000C3F19D030AD0D90501EB1220530638BFED
:10594000704700F1010008BF20F00100704700001F
:1059500050EA010C00F113801CF5000F58BFBCF594
:10596000000F01D48842704707D710F5000F58BFC9
:1059700011F5000F15D488427047894270471CF515
:10598000000F04D5BCF5000FF7D5814270474FF0EA
:10599000807C1CEB400F38BF1CEB410F01D28142D1
:1059A000704710B500F089F8922449004FF000507C
:1059B0004FF08051FFF796BE4FF47F0C1CEAD012D7
:1059C0001EBF1CEAD11392EA0C0F93EA0C0F00F0F1
:1059D000478090EA010F48BF42F480724FF0004CBC
:1059E0004CEA00204CEA012102EB0302A0FB011368
:1059F000A2F50002002918BF43F001035B0028BF95
:105A00004FEA330342EB22425FEA132C4CEBC250C5
:105A10002EBFBCEB436FB2F57C0F70474FEA036CAF
:105A2000BCF1004F08BF20F00100B2F57C0F38BF79
:105A300070470BD582F0FF0212F5803FC8BF704758
:105A400000F1C040D8BF00F00040704700F5000CE6
:105A50005FEA4C0C48BF7047B0F1C04000F073B82B
:105A600090EA010F0CEAD11348BF42F480726245FC
:105A700038BF634504D280EA010000F0004070475F
:105A800010B500F01AF800BF8900013E00F007B819
:105A900000F009B85FEA410C5FEA1C6C08D080EAAC
:105AA000010000F050B85FEA400C5FEA1C6CF6D1D0
:105AB0004FF00040A0F5800070470EF1020E2EF06E
:105AC000030E5EF8044B244204D44FEA4102B2F1C3
:105AD0007F4F11D84FEA4003B3F17F4F0CD80ED15E
:105AE0004FEAD07CB2F17F4F0CEB4C0C0CF1020C66
:105AF00008BF4CEBD17C04E04FF0080C01E04FEA0A
:105B0000D17C0CEB4C0324FA03F404F00704B4F149
:105B1000040C06D20EEB840CBDE810404CF0010CD6
:105B20006047DFE80CF0070802024FF00040A0F5E4
:105B3000800010BD0846420018BFD2F1807288BFB5
:105B400000F0004010BDFF2141EAD050C005704771
:105B500051EA000C00F113801CF5000F58BFBCF592
:105B6000000F01D48142704707D711F5000F58BFCD
:105B700010F5000F15D481427047894270471CF51B
:105B8000000F04D5BCF5000FF7D5884270474FF0E1
:105B9000807C1CEB410F38BF1CEB400F01D28842C8
:105BA000704780EA010081EA000180EA0100FFF706
:105BB000F8BE80F0004090EA010F7FF538AD81F02B
:105BC000004100F008B8000090EA010F48BF81F0E2
:105BD00000413FF52CAD421A04D882F00042A0EB00
:105BE000020011444FEAD0524FF07F4C1CEA410FA3
:105BF000A2EBD15318BF9CEA026F4AD04FF0004C81
:105C00004CEA00204CEA012121FA03FCB0EB0C0C19
:105C10000FD412F0FE0F36D05FEA4C001DD50012F3
:105C200040EBC25038BF70471CF03F0F18BF7047A1
:105C30000BE0A2F101025FEA1C2040EBC25038BF2A
:105C400070471CF07F0F18BF7047C3F120039940C5
:105C500014BF401E20F00100704780084FEA122355
:105C600008BF7047B0FA80FCA2EB0C02CCF1280C04
:105C700060FA0CF093EA122F04BF00EBC250704799
:105C80004FEAC3707047130A5FEADC1008BF704721
:105C9000F6E79CEA026F04D010EA5C0F08BF002010
:105CA000704710B5FFF709FF40DFF63E81F0004076
:105CB0007047FAF710BD0CF00F03092B08BF08203E
:105CC00000F059800A2B0BD0082B18BF704708BF73
:105CD0001CF0400F0AD04FF000004FF00001704759
:105CE0001CF0400F18BF4FF0004070471CF0100F21
:105CF00008D020F0704300F07F4242EAD3014FEA1F
:105D00004370704700F0604021F07F4242EA000299
:105D100001F07F4040EA727070474FF0FF0C4CF486
:105D2000E06C1CEA11531CBF9CEA030C9445C2BFF3
:105D3000DA4201EB02517047002B0DD0BCF1000F8D
:105D40000FD0002A01F00041A4BF41F0E04141F032
:105D50007F614FF00000704701F000414FF00000FC
:105D6000704750EA01334FF09B0C18BF4CF0806C29
:105D70007FF428A870471CF4801F11D01CF4E02F7A
:105D800003D06FEACC31490070474FF04050EFF339
:105D9000008222F0704242EA000282F300887047DB
:105DA0004FF000007047000048000000000C014068
:105DB00002000000080000000000000000010000D8
:105DC0008D3A000801020C0500000000354A000869
:105DD0000203010600000000414800080304020716
:105DE00000000000A54900080409030800000000A5
:105DF000094800080505050100000000514A000897
:105E000006060602000000005D48000807070703B9
:105E100000000000C1490008080808040000000054
:105E200025480008090A040D000000006D4A00081A
:105E30000A0B090E00000000DD4900080B0C0A0FD8
:105E400000000000794800080C010B000000000071
:105E5000194A00080D0D0D0900000000894A0008CC
:105E60000E0E0E0A00000000F94900080F0F0F0B7C
:105E7000000000009548000800000000000000003D
:105E800000000000000000003F4000000000000093
:105E900000003000400030004000000009000BC04E
:105EA0003D000BC03D00090018C024407FE02240A7
:105EB00031800000180024C01B000D80324001809A
:105EC00003801C4027401C800740004010006000F9
:105ED00000000000000000000000000000001F8023
:105EE000204040200000402020401F800000000093
:105EF000090006001F8006000900000004000400DD
:105F00003F8004000400000000100060000000005A
:105F1000000000000400040004000400040000006D
:105F2000000000400000000000000000002001C050
:105F300006003800400000001F8020402040204024
:105F40001F800000000010403FC000400000000023
:105F500018C02140224024401840000010802040FA
:105F6000244024401B80000002000D0011003FC0AF
:105F7000014000003C802440244024402380000055
:105F80001F80244024403440038000003000200063
:105F900027C03800200000001B80244024402440FB
:105FA0001B8000001C0022C0224022401F800000F5
:105FB0000000000008400000000000000000000099
:105FC0000460000000000000000004000A0011004E
:105FD0002080404009000900090009000900000074
:105FE00000004040208011000A000400180020003A
:105FF00023402400180000001F8020402740294033
:106000001F400000004007C039000F0001C00040E1
:1060100020403FC0244024401B8000001F802040BF
:10602000204020403080000020403FC020402040E1
:106030001F80000020403FC024402E4030C00000A0
:1060400020403FC024402E00300000000F00108090
:10605000204022403380020020403FC00400040062
:106060003FC02040204020403FC020402040000052
:106070000060202020203FC02000200020403FC0A2
:1060800024400B0030C0204020403FC02040004052
:10609000004000C03FC03C0003C03C003FC00000C7
:1060A00020403FC00C4023003FC020001F80204004
:1060B000204020401F80000020403FC0244024009A
:1060C000180000001F802140214020E01FA0000098
:1060D00020403FC02440260019C0004018C0244082
:1060E0002440224031800000300020403FC020404A
:1060F0003000000020003F80004000403F80200032
:1061000020003E0001C0070038002000380007C012
:106110003C0007C038000000204039C0060039C0EC
:10612000204000002000384007C038402000000018
:10613000304021C02640384020C000000000000050
:106140007FE0402040200000000070000C00038031
:10615000004000000000402040207FE000000000E0
:10616000000020004000200000000000001000108F
:10617000001000100010001000000000400000009F
:1061800000000000000002800540054003C0004000
:1061900020003FC004400440038000000000038052
:1061A00004400440064000000000038004402440F6
:1061B0003FC0004000000380054005400340000050
:1061C000000004401FC0244024402000000002E0E2
:1061D000055005500650042020403FC004400400F4
:1061E00003C000400000044027C000400000000041
:1061F00000100010041027E00000000020403FC005
:106200000140070004C00440204020403FC000403F
:106210000040000007C0040007C0040003C00000E5
:10622000044007C00440040003C000400000038095
:106230000440044003800000041007F004500440B0
:1062400003800000000003800440045007F00010A9
:10625000044007C0024004000400000000000640A3
:106260000540054004C00000000004001F800440F9
:1062700000400000040007800040044007C00040C8
:106280000400070004C0018006000400060001C0ED
:10629000070001C006000000044006C0010006C05F
:1062A000044000000410071004E001800600040010
:1062B0000000044005C0064004400000000000004B
:1062C00004007BE040200000000000000000FFF020
:1062D00000000000000040207BE0040000000000FF
:1062E000400080004000200020004000000000002E
:1062F000000000000000000000000000000000009E
:1063000000001FCC000C000000000000000008008E
:10631000300060000800300060000000022003FC34
:106320001E20022003FC1E200220000000000E1888
:1063300011043FFF10840C78000000000F0010844F
:106340000F3800C0077818840078000000780F84A8
:1063500010C411240E9800E40084000808006800AE
:1063600070000000000000000000000000000000BD
:10637000000007E01818200440020000000040025E
:106380002004181807E0000000000000024002404E
:1063900001800FF001800240024000000080008078
:1063A00000800FF800800080008000000001000DD8
:1063B000000E00000000000000000000000000804F
:1063C0000080008000800080008000800000000CC1
:1063D000000C0000000000000000000000000006AB
:1063E000001800600180060018002000000007F07F
:1063F000080810041004080807F000000000080452
:1064000008041FFC000400040000000000000E0C43
:1064100010141024104411840E0C000000000C18FD
:1064200010041104110412880C700000000000E038
:106430000320042408241FFC0024000000001F98EF
:10644000108411041104108810700000000007F07F
:1064500008881104110418880070000000001C0056
:10646000100010FC13001C001000000000000E388B
:1064700011441084108411440E38000000000700FD
:10648000088C10441044088807F000000000000049
:106490000000030C030C00000000000000000000DE
:1064A0000001010600000000000000000000008064
:1064B00001400220041008081004000002200220FD
:1064C000022002200220022002200000000010040E
:1064D00008080410022001400080000000000E00A7
:1064E0001200100C106C10800F00000003E00C185C
:1064F00013E4142417C4082807D000000004003C4B
:1065000003C41C40074000E4001C000410041FFCEE
:106510001104110411040E880070000003E00C182F
:1065200010041004100410081C10000010041FFCBC
:10653000100410041004080807F0000010041FFCE9
:106540001104110417C410040818000010041FFCE3
:106550001104110017C010000800000003E00C181F
:106560001004100410441C780040000010041FFCAC
:1065700010840080008010841FFC100400001004B0
:1065800010041FFC100410040000000000030001B0
:10659000100110011FFE10001000000010041FFC6D
:1065A000110403801464181C1004000010041FFC64
:1065B0001004000400040004000C000010041FFC80
:1065C0001F0000FC1F001FFC1004000010041FFC33
:1065D0000C04030000E010181FFC100007F008086E
:1065E000100410041004080807F0000010041FFC39
:1065F00010841080108010800F00000007F0081831
:1066000010241024101C080A07F2000010041FFCBC
:106610001104110011C011300E0C000400000E1CFA
:1066200011041084108410441C380000180010005D
:1066300010041FFC100410001800000010001FF8C8
:1066400010040004000410041FF8100010001E00C5
:1066500011E0001C007013801C0010001FC0103CD3
:1066600000E01F0000E0103C1FC000001004180CE8
:10667000163401C001C01634180C100410001C00A0
:10668000130400FC13041C00100000000804101C7C
:106690001064108413041C04101800000000000093
:1066A00000007FFE40024002400200000000300077
:1066B0000C0003800060001C00030000000040028A
:1066C000400240027FFE00000000000000000000C9
:1066D00020004000400040002000000000010001B8
:1066E0000001000100010001000100010000400064
:1066F00040002000000000000000000000000098A2
:10670000012401440144014400FC000410001FFC6A
:10671000008801040104008800700000000000707F
:1067200000880104010401040088000000000070DA
:1067300000880104010411081FFC0004000000F897
:10674000014401440144014400C800000000010468
:1067500001040FFC1104110411001800000000D600
:1067600001290129012901C90106000010041FFCAB
:10677000008401000100010400FC00040000010489
:10678000190419FC000400040000000000000003CC
:1067900000010101190119FE0000000010041FFC96
:1067A0000024004001B4010C0104000000001004AA
:1067B00010041FFC0004000400000000010401FCA0
:1067C0000104010001FC0104010000FC010401FCC2
:1067D000008401000100010400FC0004000000F836
:1067E000010401040104010400F80000010101FF9B
:1067F00000850104010400880070000000000070A2
:10680000008801040104010501FF000101040104E5
:1068100001FC00840104010001800000000000CCA4
:10682000012401240124012401980000000001003A
:10683000010007F80104010400000000010001F854
:10684000000400040004010801FC000401000180B0
:106850000170000C001001600180010001F0010CCA
:10686000003001C00030010C01F001000000010403
:10687000018C00740170018C010400000101018190
:106880000171000E00180160018001000000018408
:10689000010C013401440184010C000000000000DF
:1068A0000000000001003EFC400240020000000029
:1068B00000000000FFFF0000000000000000400298
:1068C00040023EFC010000000000000000006000EB
:1068D00080008000400040002000200000000000F8
:1068E00000000000000000000000000000000000A8
:1068F0000000000000000000000000000000000098
:106900000000000000000000000000000000000087
:106910000FFF0000000000FFFFF000000003FFFF7A
:10692000FC00000007E0007E0000001F00000F8058
:1069300000001800000180000030000000C00000CE
:1069400060000000600000400000002000004000E7
:106950000000200000400000002000004000000077
:106960002000006000000060000020000000C00067
:106970000038000001C000001E0000078000000F6A
:10698000E0007E00000003FFFFFC00000000FFFFAE
:10699000F0000000000FFF000000000000000000F9
:1069A00000000000000000000000000000000000E7
:1069B00000000000000000000000000000000000D7
:1069C00000000000000000000000000000000000C7
:1069D00000000000000000000000000000000000B7
:1069E000000000000000000000000008000000207F
:1069F0000000080000002000000800000020000047
:106A000008000000200000080000006000001FFFD8
:106A1000FFFFE000003FFFFFFFE000007FFFFFFF00
:106A2000E000000000000060000000000000200006
:106A30000000000000200000000000002000000016
:106A40000000002000000000000020000000000006
:106A50000000000000000000000000000000000036
:106A60000000000000000000000000000000000026
:106A70000000000000000000000000000000000016
:106A80000000000000000000000000000000000006
:106A900000000000000000000001E0000003E00032
:106AA00003E000000FF0000EE000001FF0001CE00B
:106AB00000001FF00030E0000030600060E00000E7
:106AC000200000C0E0000060000180E00000400005
:106AD0000300E0000040000600E0000040000C0061
:106AE000E0000040001800E0000040003000E0003E
:106AF000006000E000E000003001C000E000003C69
:106B00000F8001E000001FFF0003E000000FFE0007
:106B10000FE0000003F0001C000000000000000077
:106B20000000000000000000000000000000000065
:106B30000000000000000000000000000000000055
:106B40000000000000000000000000000000000045
:106B50000000000000000000001E00000007800090
:106B60003F0000000FC0003F80000011C0001CC0AB
:106B70000000200000004000002000000020000075
:106B80004000000020000040008000200000400085
:106B900080002000004000800020000040008000B5
:106BA0002000006001C000200000600140004000A3
:106BB0000030036000C000003C0E3001C000001F28
:106BC000FC3C078000000FF81FFF00000003E00FEF
:106BD000FE000000000001F80000000000000000BE
:106BE00000000000000000000000000000000000A5
:106BF0000000000000000000000000000000000095
:106C00000000000000000000000000000000000084
:106C10000001800000000000038000000000000E62
:106C2000800000000000388000000000006080004C
:106C300000000001C080000000000700800000008C
:106C4000000C008000000000300080200000006088
:106C500000802000000180008020000006000080ED
:106C60002000000C0000806000003FFFFFFFE000FC
:106C7000007FFFFFFFE000007FFFFFFFE00000005C
:106C80000000806000000000008020000000000084
:106C90008020000000000080200000000000802014
:106CA00000000000000000000000000000000000E4
:106CB00000000000000000000000000000000000D4
:106CC00000000000000000000000000000000000C4
:106CD0000000000000000000003C000000003FE059
:106CE0007F0000007FFFE07F8000007000C03880E0
:106CF00000007001800040000070030000400000B0
:106D000070030000200000700600002000007006E4
:106D10000000200000700600002000007006000047
:106D200020000070060000200000700700006000D6
:106D30000070030000C000007003C001C0000070BC
:106D400001F00F8000007000FFFF00000070007F66
:106D5000FC00000000000FF0000000000000000038
:106D60000000000000000000000000000000000023
:106D70000000000000000000000000000000000013
:106D80000000000000000000000000000000000003
:106D900007FF80000000007FFFF800000001FFFFF8
:106DA000FE00000007E0703F0000000E00E00780DA
:106DB000000018018001C0000010030000C00000A6
:106DC00020030000600000200600002000004006B4
:106DD00000002000004006000020000040060000E7
:106DE0002000004006000020000040070000600076
:106DF000007E0300004000003F03C000C000001FF1
:106E000001F0078000000E00FFFF00000000007F7F
:106E1000FC00000000000FF0000000000000000077
:106E20000000000000000000000000000000000062
:106E30000000000000000000000000000000000052
:106E40000000000000000000000000000000000042
:106E5000000000000000038000000000007F000030
:106E6000000000007C00000000000078000000002E
:106E70000000700000000000007000000000000032
:106E80007000001FC00000700001FFE000007000F3
:106E90000FFFE0000070003FFFC000007001F8002D
:106EA0000000007007C000000000701E000000001D
:106EB000007078000000000071C000000000007742
:106EC0000000000000007E000000000000780000CC
:106ED0000000000060000000000000000000000052
:106EE00000000000000000000000000000000000A2
:106EF0000000000000000000000000000000000092
:106F00000000000000000000000000000000000081
:106F10000001F800000003F007FE0000000FFC0F66
:106F2000FF0000001FFE1E038000001C3F3801C050
:106F30000000300F7000C000002007E0004000009B
:106F40006003C0002000004003C00020000040019A
:106F5000C0002000004001E0002000004000F000E0
:106F60002000004000F0002000006001F8006000F8
:106F70000020013C0040000030033E00C000001C27
:106F80000E1F838000001FFC0FFF0000000FF8079A
:106F9000FE00000003E001F8000000000000000017
:106FA00000000000000000000000000000000000E1
:106FB00000000000000000000000000000000000D1
:106FC00000000000000000000000000000000000C1
:106FD000FF000000000003FFC0000000000FFFF0F2
:106FE000070000001E01F00FC000003800780FC03D
:106FF000000030001807E0000060001C0060000086
:1070000040000C0020000040000C00200000400068
:107010000C0020000040000C0020000040000C008C
:1070200040000040001800C000002000380180002F
:1070300000300030038000001800E01F0000000F47
:107040000183FC00000007FFFFF000000001FFFFCC
:10705000C0000000003FFC00000000000000000035
:107060000000000000000000000000000000000020
:107070000000000000000000000000000000000010
:1070800088104FE000109FD09510D510BFD0B510DC
:10709000D5501FD0001000000080010006001FFF27
:1070A000E0080810082008C00B00FFFF0B0008C014
:1070B000082008100808000000003FFC24882488ED
:1070C00024883FFC00007FFF4482448447E04498CA
:1070D00044847C82008F000000003FFC21082108CE
:1070E00021083FFC00000800088008600802080131
:1070F000FFFE08000800000000001FFF8000600085
:1071000000000FF84888488848884FF8400040023F
:1071100040017FFE0000000000810081088288821B
:107120006884088808B00FC008B008882884C8821E
:107130000882008100810000082008C00B00FFFFCA
:10714000090008C100067FF84000400040007FFCB5
:1071500000020002001E000000042004200420049D
:107160002004200420043FFC2004200420042004E8
:1071700020042004000400000080010006001FFF1E
:10718000E00002000C00F0001FFF111011101110A0
:107190001110101010000000082008C00B00FFFFA5
:1071A0000900289127D2F554255825702558F55403
:1071B00027D2201100010000080008040906090474
:1071C00009FC0908090808080800FFC00830080879
:1071D00088046802081F0000082008C00B00FFFF99
:1071E000090008C8043044C04402440147FE44007A
:1071F00044804460041800000020402030FE070056
:10720000020004001FFFF244124492447FFC124427
:107210001244124410040000400047C2444144425A
:107220007C7C000201E27922492249224FFE492258
:107230004922792A01E70000000008010802080439
:1072400008180860FF800800080408020801080206
:107250000FFC00000000000000041FC61084FFF8AF
:1072600010881F9C0108090832A8EAA825FF2AA84F
:1072700032A821080108000000003FF02020202053
:107280003FF0000000083FC820486848A648204A50
:1072900021493F42007C000001100110792F49294B
:1072A00049494949798F07000180794F4D494B2958
:1072B0004929791F011000000200420033FE00043A
:1072C00000084100493F49224F22792249224922A0
:1072D0004F3F41000100000020002000249F249225
:1072E00024922492A492649224922492249224922E
:1072F000249F20002000000002000200420033FC16
:1073000000090211050279C2413441084114796231
:1073100005820401040100000002E802A802ABFE9D
:10732000AAAAEAAAAAAABEAAAAAAEAAAAAAAABFED4
:10733000A802E80200020000000000000FF0082090
:10734000082008200820FFFF082008200820082027
:107350000FF000000000000020212021202223E265
:10736000F224222822302FE022302228F22423E2A5
:107370002022202120210000008007000000FFFFC4
:1073800008000408103011C11E22F0C4101817E0C4
:107390001018104611810000040108091009EF922D
:1073A0002AB22AEA2AA42AA42AA42AAA2AB22FA202
:1073B00020012001000100007E9752904A967FE054
:1073C0004AA652A07EAD0402040C0470FF80047033
:1073D000440C34020401000002000200420033FCAD
:1073E000000900120004001800E0FF0000E000188F
:1073F00000040002000100000081008108828882F0
:107400006884088808B00FC008B008882884C8823B
:107410000882008100810000020002004200420058
:107420004200420242017FFE42004200420042000E
:107430004200020002000000000808100820084076
:1074400008900B100C10FFFF0C100B100890084058
:107450000820081000080000082008C00B00FFFFEB
:10746000090008C100067FF84000400040007FFC92
:1074700000020002001E000002000202420433F873
:1074800000040002FFFA9212922293029282924228
:10749000FEA2011A000200000000003E3E020202AD
:1074A000020202020202FFFE0202020202020202C3
:1074B0003F02003F000000000080010006001FFFA7
:1074C000E00002000C00F0001FFF1110111011105D
:1074D0001110101010000000040804102420244093
:1074E00024FF2492FD92269224922C92149224FF3F
:1074F00044000400040000000000000000007FFFC2
:1075000041024102410241024102410241027FFF28
:10751000000000000000000000112012FFF4249081
:1075200024902498FFF52012000C7FF04440444240
:1075300044417FFE0000000000017FFE04800480C3
:10754000FCFF040100063FF824012782246444184C
:10755000C4644782000100000008081008200840A9
:1075600008900B100C10FFFF0C100B100890084037
:1075700008200810000800000808493049FF7F2251
:10758000492249227F3F08009010511031101FFFFF
:1075900031105110901000004020422245445AA85A
:1075A0004920EAA24CA140BE5CA0EAA049204AA81A
:1075B0004C84404240400000010041004100410035
:1075C00041004102410147FE450049005100610070
:1075D00041000100010000000200420033FE0004EF
:1075E000000822002AFF2AA82AA8FEA82AAA2AA957
:1075F0002AFE220002000000082008C00B00FFFF46
:1076000009000A8204220A1A3282C27232060A1A57
:1076100004E202020202000002022202240225FA0F
:10762000295231522152FF5221523152295225FA08
:1076300024022202020200000040004024402440B4
:107640002440244224413FFE444044404440C4403E
:107650004440004000400000082008C00B00FFFF2D
:107660000900088047FF4410442044C07F00448044
:107670004462440147FE0000000000002004002096
:107680000C1020180E2010063FE00000100000082B
:1076900000000C21FFF421220421220629220625C4
:1076A000220627FFF6272206292206292206312252
:1076B0001611223E01FFF600000400000000000049
:1076C00004000008000000000000000200010000AB
:1076D000100000000000000004FA97999999D93F22
:1076E000AF788E1DC571CC3F9FC678D0099AC33F35
:1076F000935555555555E53F599322942449D23F0A
:10770000DE03CB966446C73F44523EDF12F1C23FD0
:10771000000000000000000002400000000000A087
:107720000000000005400000000000C8000000004C
:107730000C4000000000409C0000000019400000C8
:107740000020BCBE0000000034400000BFC91B8EFA
:1077500000000004B5400000504BCFD06607E2CFD8
:10776000010000006C4100003E8251AADFEEA73408
:1077700001000000D9420000DCB5A0E23A301F97BA
:10778000FFFFFFFFB4450000FD25A0C8E9A3C14FDE
:10779000FFFFFFFFFF3F000000000080000000002F
:1077A000FF3F00000000008000000000E8770008B4
:1077B00000000020B005000028010008F079000852
:1077C000B0050020900F0000840100081C0000009C
:1077D00043000000F8FFFFFF0C0000000E00000057
:1077E0000F0000002E000000011184A24A04680965
:1077F00001020304060708090C69101502040608B3
:1078000014F07F451008E076453313954314B01A01
:1078100046041A401C46481D7FF8FFFCC00CC20CF1
:10782000C70CC38CC1CCC1CCC38CC70CCE0C9C0C78
:1078300039FC13F81C1018C84CDCECCFCCC78CC733
:107840008CCFCCDCECC84CC00CFFFC7FF8601A90ED
:1078500002680B67E01FF8300C20044002023D2054
:10786000047808961008F007F80FF81BFC2014FCA9
:107870001FFC3FFC7FFCCFFC03FC1CFC2FF803F833
:1078800001F0100D03C00FF01FF838FC603C401EE3
:10789000100C1E188E1B8E1F8C1D8C119812106AD6
:1078A000209429721808C48CDFECDFECC40A4BC7A3
:1078B0008C78491C4811C3CCCFECC96CD92CD12C85
:1078C000D36CDE4CCC0C1C1401010E120E2B03F8F1
:1078D00070180EE3FCC3FCC3CCC204C204C3CCC307
:1078E0000E1A7F861303F80AAAFF015BFE2F080A0F
:1078F00015AF08DA8F301A0F051AE3080A15EF08DA
:1079000059203901A9105920B90822E06A3F0829F5
:107910003019082A3E3029085918E9080A153F602D
:1079200039B00912086970E9305ADFD049082BFED6
:107930003E083EE3FFFC3E2F083AF8903CE3FFF0A0
:10794000905CE3FFE0105AC0104B803E10114908D4
:107950005AFE084AFCC04CE3F802304BF006503C9B
:10796000E00E3E904BC01E083B803E0812E05A7E5F
:10797000F03AFE305BE001085A03083B07FE404C3A
:10798000E00FFE305A1F082C3FFE7E0819B85BFE40
:107990008FDC3930213988A9084960F918496059C4
:1079A000203EE3FF063EDFC84A0E084BFC1E084B94
:1079B000F83E204BF07ED04BE0FEE85AC1084B83E6
:1079C000FE2019A8091A6099105A7E103BFEEF0894
:1079D0003A010829C969082920990169106AFE102D
:1079E000E908D930098101013B09123CB2080000C5
:04000005080001E905
:00000001FF
